:020000041100E9
:10300000002373B52B4D2C4C28006361022601F080
:103010005BFA4021FE2221742800284B009601F023
:10302000A5FA002836D1217CFF222800244B0096E7
:1030300001F09CFA00282DD1224BA2899A4226D178
:10304000E389214A93420DD1204B6361204B2268D2
:10305000002A03D1002B01D043CB43C4280001F048
:1030600071FA73BD1B4A934201D00023EFE71A4B5C
:103070001A4A1B68934206D9C02304222800217CE7
:103080009B0001F0E9FA114B6361154BDFE7002368
:103090002374EAE7CC233821AC2228009B01217459
:1030A00001F0DAFA0028F2D10E4B63610E4BE38196
:1030B0000E4BCCE7BC44FF1F6064FF1F6C64FF1F16
:1030C0006E64FF1F5959000083050000F54200118E
:1030D00050BB0011821500008464FF1F871300009D
:1030E0005CBB0011AD430011AAAAFFFF44BB001155
:1030F000F7B5164B0192C318021D002000938823D8
:103100005B05D3181B685C1C1AD09CB2402C18D8E5
:103110008D781E0CAC466746CD782D023D43AE42FD
:1031200006D1019800280ED110000C70240A4C70B2
:1031300003249BB20733A343D218009B9A42DED3E9
:10314000FEBD4432F9E71000FAE7C046FC0F00006C
:10315000802213B503000324019189B25201073183
:103160009B18A14304305A1A88235B05C3181B68B7
:10317000591C03D190429241104016BD99B240298A
:1031800007D80B000733A343C0189042ECD30020AC
:10319000F3E74430F9E7134B134A1B68126810B584
:1031A000FA24934201D81A00F824104BE4021B6859
:1031B0009A4210D813000E4A12689A420ED3013375
:1031C00007D1F823DB029C4203D10A49054808F0E5
:1031D0001FFC200010BDFC24E402ECE7FE24E40206
:1031E000F7E7C04600C0071100D0071100E0071143
:1031F00000F00711FFFFFF7FF0B59BB015000490B2
:103200000391402A00D9A0E006AB59801A80FFF74D
:10321000C2FF0400042816D9002206A9FFF768FFA0
:10322000052810D906AB1B88AB420CD1002D07D066
:10323000514B2A000499C01808F092F9002802D1D5
:1032400001201BB0F0BD06AB1D8020000699FFF7E2
:103250007FFF041E7BD1069B0793FFF79CFF802313
:103260005B01C618802307001B039E4201D3F8268A
:10327000F60288235B05F31801931B68013302D023
:10328000019808F00DF93D49019808F0C1FB3B1D7C
:103290000293331D05938822029B52059B181B68DD
:1032A00008935A1C3CD044219AB20091402A04D879
:1032B0000320D11D814389B2009103991B0C8B42DD
:1032C00024D0402A22D80122300008A9FFF710FF9D
:1032D000021E1BD1380008A9FFF70AFF04000428CA
:1032E00031D9009A059B9B1880225201B218934253
:1032F00040D288235B05C118009A09A808F060F93C
:103300001D4B009A09A9F01808F0B2F9009A029B27
:103310009446634402931A4B029AFB189A42BAD31A
:1033200088235B05FC1821680198013908F070FBBF
:10333000200008F0B5F8039A07AB5A8030000799CF
:10334000FFF706FF0400002C03D1002079E70428D2
:10335000FBD988235B05E018069908F059FB032385
:10336000EA1C9A4300D16BE7034B0499E01808F07C
:103370007FF965E70424ECE704000011FFFFFF7FFD
:10338000F80F0000F7B505001400402A21D80027E7
:1033900001AE71803780FFF7FEFE042816D93A008F
:1033A0003100FFF7A5FE042810D93688BC420BD0A7
:1033B000BD4209D0221CB44200D9321C064B92B245
:1033C000C118280008F0FCF830B2FEBDC04300B2BE
:1033D000FBE703204042F8E70400001137B5042260
:1033E00004000D0001A81649FFF7CCFF02000428D5
:1033F0000BD1019BA34208D3AB4204D0104901A8D2
:103400000195FFF7F9FE01203EBD0E4C2368200018
:10341000019308F045F8019920000139019108F065
:10342000F7FA80235B01E418074B9C42EED104229B
:10343000034901A80195FFF7DFFE0020E4E7C0463D
:103440005555000000C007110000081130B589B0C3
:1034500008F006FB10226946254808F0F9F9254BCB
:10346000009A9A420ED1019B029A0F2B33D8002169
:1034700001240698013B08D2002900D00292029B49
:10348000013331D10023029325E0551CF2D1020013
:103490002100EFE710341022200004A908F0D8F929
:1034A000029B013301D1069B0293882304995B059B
:1034B000C918059B06981A03120B049105928142C4
:1034C00003D02B4201D108F07BF8019B013B019313
:1034D000019B002BDED1029B002B03D004930498A8
:1034E0004168084709B030BDE025014C2D03EFE7E6
:1034F0000000011150485936F7B50F4F0F4BFA6DC8
:1035000004001A4084235B001343FB65030010335F
:10351000019300252E00112008F052F90322BB6E02
:103520001340AB4002351E43202DF4D1019B40C413
:10353000A342EED1F7BDC04600F0004000FEFEFF02
:10354000802270B5AD4CAE4BD200002120001C6033
:1035500007F066FF2300AB4A88331A60AA4B1A783B
:103560006E23002A00D01133E3620A232365A74BA0
:103570001878A74BA0630138E361C3B2032B01D8CD
:1035800010232362A34B37226361C823DB00A361AE
:1035900023008C331A60082336210F3AE518E163C3
:1035A00023646264E9670439251DE96725003B2629
:1035B000BC352E602500C0352B602500C4352A603F
:1035C00025000636CC352E602500083EC8352E6015
:1035D0002500D03529602100D4310B602100D8317D
:1035E0000A6021000225E0310D6025004221DC3512
:1035F000296025001B3EE4352E602500E8352B6050
:103600002500EC352A6022000525F43215602200E1
:10361000F032116022001831903211602200943291
:10362000136023003C2298331A60AF23DB00236031
:10363000794B2363032805D807F0AAFF33023537F7
:103640001523636096232100FA225B00A360E360E8
:10365000C8332361714BFC319200A3640A6062623B
:103660006F4A704DA2627322E2656D3A6265A2658F
:103670000232E5644A600221616696218900A166F2
:10368000626709210022E166A2676749674A684EBE
:103690002167E2673560032811D807F079FF9608A3
:1036A0009EA61023CDE70E23CBE70C23C9E720000D
:1036B0001A259C30056020000735A03005602000E9
:1036C000A83003602300FA20F8338000186023003C
:1036D0006420A433186023005F38AC3318602300E3
:1036E0000338B03318602300C630B43318602300A9
:1036F0000020B833186023003825FC339D604D4D01
:103700005A665D644C4D9A64DD619625AD001D627C
:103710004A4D9A675D62F53DFF3D9D621E25484A10
:10372000DD6618675867D9651966DA67BE23C02158
:10373000444A5B00E250444B4900635004316250FC
:10374000C4225200A350FA23E4205B000432A350A9
:103750000432A3503D493E4A3E4BD1603E49800071
:1037600019503E49E938FF3819503D490430195085
:103770003C491038D1613C4911633C4951633C4993
:1037800011603C49195019003B48F83108603B4929
:10379000D16582213A4A89005A501A0039490832C3
:1037A000D1671A003849B43211608821374A89003C
:1037B0005A501A00364988321160364ADA6407F0E6
:1037C000D7FF012007F01CFF70BD200014259C309E
:1037D000056020000435A03070E7200010259C30E3
:1037E000056020000335A03068E720000E259C30DE
:1037F000056020000235A03060E7C0460004FF1FCE
:103800003067FF1F2072FF1FF446FF1F4A0AFF1F89
:103810003A07000080C3C9019A02000050C30000AB
:103820006A180000280A0000204E000088130000DB
:10383000F009FF1F001F001168100000C4090000FC
:10384000DC05000040420F0010270000FD1BFF1F99
:10385000FC00FF1F0000FF1F012FFF1F2932FF1F69
:10386000C130FF1FD51FFF1FF11FFF1F9D21FF1F2D
:10387000491FFF1FC128FF1F692CFF1FD918FF1FF9
:10388000CD27FF1F3525FF1F4125FF1F491EFF1FA5
:10389000011FFF1FC11DFF1FF7B50B0CFF270122E2
:1038A000009300233C001E001D009446019089B245
:1038B00062469A401000084018413618B6B2FF2FF1
:1038C00002D1012E00D19FB2009802401A41AD18DA
:1038D000ADB2FF2C02D1012D00D19CB20133102BCF
:1038E000E6D10320012E07D1012D04D1019B240133
:1038F000E4191C700138FEBD102EFCD10238102DC9
:10390000F9D00230F7E710B5064C2378002B07D129
:103910000548FFF7F1FD0548FFF7EEFD0123237091
:1039200010BDC046F066FF1F0467FF1FF466FF1F4F
:10393000F0B58BB00D0001230190102936D8FFF7A8
:10394000E2FF00231A001B48C15C01335218102B00
:10395000FAD1023B002A29D0174B184C1F680023CC
:1039600006A9E25C1600FA5C56405E540133102B47
:10397000F7D102AA07F03CFF2A0002A9019807F03C
:1039800067FD07F0FDFD23681B18236007F0F8FDB5
:1039900063681B18636007F0F3FDA3681B18A3603E
:1039A00007F0EEFDE3681B18E360002318000BB07E
:1039B000F0BDC0460467FF1F9445FF1FF466FF1F5C
:1039C0000223F0B50124614D614E2B70614B91B023
:1039D0001C70614F03933368002104207B7006F054
:1039E000DFFB042006F0D6FA0023984205D07A784F
:1039F000552A02D0332A00D09BE03360002006F025
:103A000049FD07F095FFFFF79BFD07F069FD1F22B9
:103A100001240021514B10AE1A70514B1C70514BB8
:103A20001970514B19689143163A0A431A60602283
:103A300019689143403A0A431A6007F0B9FE07F04B
:103A4000C7FEC120FF21494B80001A588A431A50F3
:103A5000C522920098588843BF390143995098581D
:103A6000434908408021C901014380209950995859
:103A7000C0050902090A0143995080213D484901C6
:103A800007F016FD032322003B49019400933B48B5
:103A900007F076FF2C223A4905A807F091FD05AC06
:103AA00061782078023406F095FAA642F8D1354CB8
:103AB0001120002106F0A2FB2268334B03201A409C
:103AC000A023DB0213432360802322689B0413435B
:103AD000236022682D4B1A4080239B0313432360ED
:103AE0002B4A2C4B934200D8012007F0C1FE07F06F
:103AF0003FFF80232268DB0413432360287807F00C
:103B000027FD039B1878C0B207F01AFD07F0F8FDF7
:103B10002149042007F0FCFE06F088FC00F0B4F810
:103B200000F0C6FD00F058FE00F010FA002011B0C1
:103B3000F0BD00932100184A042007F049FF8023BC
:103B4000DB059C62FFF782FC58E7C0464A0AFF1F6C
:103B500034F00040F446FF1F9064FF1F480AFF1F27
:103B6000490AFF1F680AFF1FBCF0004000E100E0A7
:103B7000FF00FFFFF846FF1F7C59FF1FF856FF1F8D
:103B800070BA001114F00040FF7FF8FFFFFF9FFFA5
:103B90000080FF1F2072FF1F3B00010870B5002549
:103BA0002A492B4A2B484D6308CA1B051B0DED18EB
:103BB0008242F9D10022284B8B63284B08211A62DC
:103BC0008022274B9205DA67264BDA688A43DA604F
:103BD000254A1278012A03D09A6824490A409A603B
:103BE00000260121224C11202660DA688A43DA601F
:103BF00007F05EFD112007F0F3FB8022636C934316
:103C00006364EE24E4006C431A4A200C040064232D
:103C100090420AD8FA223300D200904205D9164BBE
:103C20000A21C01807F0E4FCC3B2144A1120137231
:103C3000D48007F0ADFD124B1B78002B04D1114B43
:103C40001021187807F0ACFC70BDC046000005409C
:103C50008805054000060540FF01000000F0004017
:103C600004E100E03CF000404A0AFF1FFFDFFFFFD5
:103C700000380040B70B000030F8FFFF7864FF1FEA
:103C8000B266FF1FB064FF1F002210B511001120A3
:103C900007F0A6FE10BD0000F8B500230125082698
:103CA000344F354C3B62E3681120AB43E360E3687B
:103CB000B343E36007F094FB112007F0F9FC1120F7
:103CC00007F07EFE402322681120134323608023E7
:103CD0006268DB02134363608023A2681343A3601E
:103CE000A368264A1340A3608023A2689B01134364
:103CF0001022A360236C93432364236C2B4323641F
:103D000080235B003B62226B1D4B1A402263626B77
:103D10001A406263A26B1A40A263E26B1340E36332
:103D2000E368184A1340184AE36013682B43136092
:103D300007F06EFBFD21154B154A89005A50802370
:103D4000C720626B5B0313436363E3688000334304
:103D5000E360E3680F4A1D430F4BE56019581140BB
:103D6000802212020A431A50802292051A600B4BDD
:103D70005E63F8BD00F000403CF00040FFFFDFFF55
:103D8000EFFFEFFFFFFF7FFF003800400000FF1F45
:103D90009D3B0011FF00FFFF00E100E00000054037
:103DA00030B503A804880B20002C0ED14968074DBC
:103DB00008784978090201430A20A94205D1012166
:103DC00020001980024B1B7A137030BD192A0000A5
:103DD0007864FF1FF7B5150008AA16884A680F4FC8
:103DE00014785278120222430A24BA4214D10122D2
:103DF000DBB2019200962A0007F068FA041E0BD18C
:103E0000074B1B68002B07D068782A780002104304
:103E100042425041013098472000FEBD0229000077
:103E2000FC63FF1F30B5012503790400BFB02B42AE
:103E300012D00A49408806F0B5FD28420CD06A46E7
:103E4000074B69465B8D55801380064B60881B7A53
:103E50001371002203F086FE3FB030BDF463FF1FF4
:103E60003043FF1F7864FF1F10B50549054806F071
:103E70004FFD0421044A054806F00CFD10BDC04664
:103E8000F463FF1FFFFF00009CBA00113043FF1FC7
:103E900010B5024804F0E8FC10BDC046253E0011F4
:103EA000062310B5837010330371443B43712A33EA
:103EB00083714433C37100230222012103720E4B2C
:103EC000027041701C8881724472197A0273C17247
:103ED0009A784273DA7882730322C2731A79027471
:103EE0005A7942740C2282749A79C274DB79037510
:103EF0001123C370152010BD7864FF1F10B5122068
:103F000007F096FC104B12220021186007F088FA87
:103F1000002007F035FC012007F04AFB022003F0E7
:103F200047FF032005F05CFF042003F085F905201E
:103F300003F052FE062001F0E7F9072006F08AFCA4
:103F4000082000F0D1FF10BD0064FF1F10B507F07E
:103F50003FFB012007F0A4FC07F0FAFC002010BD95
:103F6000094B10B50400984205D0012904D1200066
:103F7000064906F0CDFC10BD0229FCD1013904F040
:103F800031FC0028F3D0F6E7FEFF00002664FF1F97
:103F900070B50D7A100004AA2C0016881022144067
:103FA000154220D1002E20D10A78022A18D14A6861
:103FB000517815780E4A09022943914205D00D4ADD
:103FC000914209D01C800A2404E014220A491A8074
:103FD00007F0F6FA200070BD0C2208491A80F7E7B6
:103FE0001C800124F6E70824F4E70B24F2E7C0461E
:103FF000F3FF0000F4FF00007845FF1F74BB0011C1
:1040000010B504000749084806F082FC074804F090
:104010006BFB0020E40704D50721054A054806F09C
:1040200039FC10BD2664FF1FFFFF0000613F001137
:10403000DCBA00117443FF1F00B50C4BBFB01A78F7
:104040000B4901A800F082FC6B4680B25880002822
:1040500009D06A46074B69461B881380064B00222D
:10406000188803F07FFD3FB000BDC0460464FF1F09
:104070000564FF1FCE43FF1FD844FF1F00B50C4B44
:10408000BFB01A780B4901A801F0B2FC6B4680B2B0
:104090005880002809D06A46074B69465B8D13801B
:1040A000064B0022188803F05DFD3FB000BDC046FE
:1040B0002E64FF1F2F64FF1F7443FF1FD844FF1F90
:1040C000F7B50E00377A1C0008AB11003D001A88C6
:1040D00020231D401F423CD13378022B3BD1736813
:1040E0001F785B781B023B431E4FBB4208D01E4F1C
:1040F000BB4214D01D4DAB4221D00A252800FEBD85
:10410000002A2AD1142C2AD82200F06807F058FA85
:10411000174B1C70012CF1D9FFF7B0FFEEE7002A16
:104120001BD1202C1BD82200F06807F049FA114B54
:1041300004211C70104B187807F032FADEE7E3B266
:104140000124009201940A00310007F0BFF8050035
:10415000D4E70825D2E70125D0E70B25CEE70D25CA
:10416000CCE7C046F3FF0000F4FF00000229000086
:104170002E64FF1F0464FF1FB064FF1F332310B5BC
:10418000040003700A220749013007F019FA064BB0
:104190000F201B681A0AE37222731A0C1B0E62733B
:1041A000A37310BD7864FF1FA064FF1F30B5012505
:1041B00003790400BFB02B4213D00B49408806F0AE
:1041C000F1FB28420DD06A46084B01A81B881380DA
:1041D000FFF7D4FF6B46588000226946608803F0E1
:1041E000C1FC3FB030BDC0462664FF1FCE43FF1F59
:1041F00010B5024804F038FB10BDC046AD410011B7
:1042000070B5160004AA148805AA15784A68507873
:10421000117800022A4A0843801805284BD807F075
:10422000B7F903131E29343F0720032C0BD80422AF
:10423000121BAA4200D92A0022491A80300009190B
:1042400007F0BEF9002070BD0720112CFBD8122208
:10425000121BAA4200D92A001B491A80EEE7072048
:104260000E2CF0D80F22121BAA4200D92A0017499F
:104270001A80E3E70720032CE5D80422121BAA4288
:1042800000D92A0012491A80D8E70720032CDAD86F
:104290000422121BAA4200D92A000E491A80CDE737
:1042A0000720032CCFD80422121BAA4200D92A00CF
:1042B00009491A80C2E700220A201A80C3E7C046D3
:1042C000DCD5FFFF27BB00114C64FF1F17BB00119B
:1042D00012BB00110DBB001108BB001110B50D2160
:1042E000024A034806F0D6FA10BDC046FCBA0011D7
:1042F000E443FF1FF0B50024274E85B03000B471B1
:1043000000F0E2F8254D264BEA89297C9A422FD10C
:104310000423300003AA00F057F90400300000F035
:1043200011F90123B371002C34D16B4699892B68A4
:10433000C9BA4B4329891B4A1B145B1853806B462F
:10434000D9896B6849BA89B24B4369891B0C5B18E0
:104350001548191C1BB2834200DD011C0B0400D55B
:1043600000211388918001331380200005B0F0BD37
:104370000227220003AB3000009700F0F7F80E236D
:104380000400297C0122300000976B4400F0EEF815
:104390000443C3E71C00E8E7BC44FF1F6064FF1F41
:1043A000830500007864FF1F0F27000073B5234EBC
:1043B000300000F089F8224D07236A463000297C3E
:1043C00000F002F904003000002C33D16B461B785A
:1043D0007F2B2FD800F0B6F86B46D878F023020474
:1043E0001B031A406B469B8816495BBA9BB21A4363
:1043F0002B68000953432A891B0C9B184B806B4682
:104400005A789B7812031B011A436B68024353438B
:104410006A891B0C9B180C481A1C1BB2834200DDD6
:10442000021C130400D500220B888A8001330B8004
:10443000200076BD00F086F80124F9E7BC44FF1F98
:104440006064FF1F7864FF1F0F27000070B5114CD8
:10445000237C002B0FD0382B0ED10F4D280000F0FD
:1044600033F8CC23AC222800217C9B0100F0F4F827
:10447000280000F067F870BD084BE2899A42FAD133
:10448000054D280000F020F800222800217C00F0D3
:10449000C5F8EDE76064FF1FBC44FF1F8305000003
:1044A00010B5084B1A7C002A09D05B69002B06D096
:1044B0009847041E01D0FEF7A3FD200010BD012483
:1044C000F9E7C0466064FF1F70B5C17905000C00B4
:1044D000631E9C411A4BE402E41849000460C9B20F
:1044E000007905F0C1FEE979687949000131C9B266
:1044F00005F0BAFEE8790930C0B207F061FA00238E
:10450000E36661332360AA795B3B002A0ED0226800
:104510009A43023B134323600A23E3610733236278
:1045200000232363A3630133E36370BD22689A43CE
:10453000022313432360462363610633A361EFE73D
:104540000050004070B5002504000368DD66C079A6
:104550000930C0B206F044FF2900207905F020FEA2
:104560002900607905F01CFE70BD0000F8B51E0042
:1045700006AB1D78002304681700E366616007F04E
:104580006FFA01238022E3662B0027615200013B72
:1045900008D206F075FF08200A4A1168002D03D1E1
:1045A0002800F8BD2261F2E7236F034203D023699C
:1045B000013D3370013613685B1A032BEED90125D8
:1045C000EEE7C0466008FF1F70B51C0000230568B9
:1045D0001600EB66696007F043FA01238022EB6660
:1045E00023005200013B08D206F04AFF08200A4A85
:1045F0001168002C03D1200070BD2A61F2E72B6FF7
:10460000034203D02B69013C3370013613685B1AF7
:10461000032BEED90124EEE76008FF1F002370B5DD
:1046200004681500E366616007F01AFA0123E36687
:10463000256106F025FF8020064A80001168636B23
:10464000034205D113685B1A032BF8D9012070BD12
:104650000020FCE76008FF1F70B51D000023046800
:104660001600E366616007F0FBF90123E36626614B
:104670000F33626B1A42FCD02B0A23611023626B4A
:104680001A42FCD0EDB2256106F0FAFE8020074AFE
:1046900080001168636B034205D113685B1A032B1A
:1046A000F8D9012070BD0020FCE7C0466008FF1F5C
:1046B00010B5084CE368002B08D1074B1B685B045E
:1046C0005B0C0A336360054B1B68236007F0A8F896
:1046D000A06010BDA064FF1FC8F00040CCF00040F7
:1046E00010B507F0BDF90F4B996A9A6A8A42FBD15F
:1046F0000D4C6268A0688A18121A531E884200D3B3
:104700001300A1602168DA0B52185B0407495B0CA7
:10471000636022600B60064B1A6006F0B1FE2068F1
:1047200010BDC04600F00040A064FF1FC8F000406C
:10473000CCF0004070B51F4C23793F2B01D93F23AB
:1047400023711D4B22791A701878C0B206F0A0FEB2
:1047500018231A491A4A0B801A4913800B80538078
:10476000A379194980200B800C21938001334B439E
:10477000164D191C0001834200D9011C2980D180EB
:104780006379002B11D101336371237A012B01D896
:10479000022323726279237A0D4853430A21584336
:1047A00006F026FF0B4D286070BDA02BEDD9A0238D
:1047B000EAE7C0469464FF1F480AFF1FD644FF1F64
:1047C000A046FF1FD444FF1FD244FF1FD044FF1F49
:1047D000710200008464FF1FF8B513210020FEF76A
:1047E000FDFD114C011E114D09D10C22104BC1CB06
:1047F000C1C4280006F014FEFFF79CFFF8BD0C2290
:1048000020000C49FEF7BEFD0C2802D0084B43CB1C
:1048100043C40C2228000849FEF7B4FD0C28EBD055
:104820000C220021E5E7C0469464FF1F6064FF1F6F
:1048300068BB0011FC0C0000F50C0000F0B51D4C2D
:104840008022A5440400882069465201400506F0F4
:104850008FFE902212016A441300200032C832C336
:1048600016C816C38023144C144FA6689B03334309
:10487000A3603B6006F0E4FD8823A0685B05C018D8
:1048800006F00EFE0025882329008022A0685B0523
:10489000C01840196944520006F0EAFE8023013531
:1048A000FF355B019D42EED1A6603E60044B9D4406
:1048B000F0BDC046FCEFFFFF1046FF1F9808FF1F2A
:1048C00004100000F0B5040087B0002825D0684629
:1048D00006F0DEFF1B4C022806D1062269462000A6
:1048E00006F03EFE002816D06946002301250F265B
:1048F0002F00E25C013310091030874038002F0090
:10490000324097403A0002434A610439062BEFD106
:104910006846FFF793FF07B0F0BD182269460A48C2
:1049200006F026FE6A46A300D358013305D01822AC
:10493000FF21684606F074FDEAE70134062CF1D148
:10494000E9E7C0466509FF1F00090011F0B5002521
:1049500004000E0085B0AA4200D183E04B1C087809
:1049600001934B788978377909021943F3783F0628
:104970001B040B431F43039720706570252800D14B
:1049800093E033D8112813D806F072FD66000D01AC
:104990000D010D010D01A700B500AE000D010D01C7
:1049A0000D010D010D010D010D010D01E7000701C4
:1049B000232800D1C0E0DB2800D016E1042A00D86B
:1049C000A9E01025052A05D0551F2A003800711DC1
:1049D00006F0F6FD05223100200006F0F1FD2A0068
:1049E0003900601D06F0ECFD05353BE0562856D039
:1049F00010D8332800D19AE0552836D02628DAD1AD
:104A0000894B2900132218001D0006F009FDFEF74E
:104A1000F7FA59E0712800D174E0722800D17DE0E6
:104A2000DC28C8D1022A00D875E07378BFB2637061
:104A3000B378A370032A05D0033A390092B2F01C70
:104A4000FEF7DAFB10223900E01CFEF79BFCC51CC8
:104A5000002807DA60705CE00C222000734906F041
:104A6000AFFD0C25280005B0F0BD013A704D0C2AB1
:104A700013D8002A0AD02800019906F0A1FDFFF7FB
:104A800059FE0C2228006B49FEF7B6FB29000C22C8
:104A9000601C06F095FD0D25E4E70C22EBE7644D64
:104AA000654B2A0043CB43C2E9E7013A5E4D0C2A2D
:104AB00011D8002A08D00199280006F081FD0C22A7
:104AC00028005E49FEF798FB29001322601C06F0BF
:104AD00077FD1425C6E70C22EDE705225849601C36
:104AE00006F06EFD0625BDE712225649601C06F051
:104AF00067FD1325B6E708225349601C06F060FDE8
:104B00000925AFE77178F72905D8504B188801F0CF
:104B1000CBFB0225A6E7FF236370FAE74C4B012A83
:104B200003D072781A706270F3E71B78F4E7200004
:104B3000FFF724FB050095E7042A04D9454D2F60B3
:104B400006F06EFEA860FFF7CBFD0422039003A9D8
:104B5000601C06F035FD052584E73F4D062A15D972
:104B600006222800019906F0FBFC00280ED0062240
:104B70000199280006F024FD062238492800FEF796
:104B80003BFB0123324A11780B43137029000622A4
:104B9000601C06F015FD072564E7012ABBD070787C
:104BA000FFF790FEB5E7012800D004E7931E2C4FD5
:104BB0001A2B04D87378002B09D100F009F9294B7E
:104BC00039001D78601C6A1E06F0FAFC4AE7551E83
:104BD0002A000199380006F0F3FC2349AAB23800F4
:104BE000FEF70AFB00F02AF9E9E7DA2893D1042A54
:104BF00091D9082A15D9B37972791B021343F27936
:104C000012041A43337A1B0613433B603B680522A8
:104C100031002000039306F0D3FC0422601D03A999
:104C20006CE7FE236370F1E76064FF1F74BB001143
:104C30009464FF1FFC0C000068BB0011F50C000021
:104C40006C64FF1F4C64FF1F1446FF1FD844FF1FF6
:104C50009064FF1FA064FF1F6509FF1FADAC00003B
:104C60009166FF1F8F66FF1FAEDE000070470000D9
:104C7000020010B5094B0A32094C92B2DA815A820D
:104C800098811882207802F075F90422054B0121E1
:104C900020781A7006F084FC10BDC0469E45FF1FA8
:104CA000DA66FF1FD966FF1F013870B5042809D8DE
:104CB00006F06EFC0309230812001E4B022118782F
:104CC00006F06EFC70BD1B4B0821187806F0C0FC86
:104CD0000022194B1A72F5E780220024164B154D5D
:104CE00052001A81082128781A68DC7206F098FCB4
:104CF0002100287806F054FDE4E70E4B08211878CF
:104D000006F0A6FC0D48FFF7CBF80D4B0D4A9B793A
:104D100093800D4A13800022074BDA720132FF3272
:104D20001A810A4B1B78002BCCD0094A136006F07D
:104D3000D7FDC7E7B064FF1F8464FF1FE144FF1F76
:104D40009464FF1FA046FF1FD244FF1F9064FF1F03
:104D500034F0004010B5002904D1042802D10D30F0
:104D600005F04CFA10BD000010B501290ED1042841
:104D70000CD10D3005F042FA054B1B78002B05D005
:104D80002622044B04485A72FFF772FF10BDC0463A
:104D9000B266FF1F8464FF1FC40900000300F0B562
:104DA0000A4D8E18B14202D152008018F0BD0C7825
:104DB0002F6824093C5D0F271C700C7801313C40A2
:104DC0002F683C5D5C700233ECE7C046CC44FF1FAB
:104DD0000D22114B10B51A700C23104C1049237082
:104DE000093A033B0F48637006F0EAFB2D230122CA
:104DF0000D490E48A371FFF7D1FF01220C49FFF7BF
:104E0000CDFF01220B49FFF7C9FF00220A4910001C
:104E1000FEF7F2F910BDC046AE66FF1F8F66FF1F9A
:104E200027BB00119166FF1F6709FF1F9666FF1FD2
:104E30006609FF1F6509FF1FAEDE000070B5124C4A
:104E4000132220001149FEF79DFA114D002817DDAD
:104E5000AB78002B14D0431C2B7009236B700023FC
:104E600000190370287829000130C0B206F030FD27
:104E7000297822000139C9B2002005F029FC70BD53
:104E8000FFF7A6FFEEE7C0469166FF1FAEDE00000B
:104E90008F66FF1F10B5114B1A781870002A0ED0BC
:104EA00000280BD10E4B1A78062A07D85423D3407A
:104EB000DB0703D50B4B187802F05CF810BD002817
:104EC000FCD0074B1B78012B02D0033B022BF5D8FB
:104ED000044B0121187806F063FBEFE7B266FF1F71
:104EE000D966FF1FDA66FF1F70B54D4E4D4A4E4919
:104EF0003070042005F078FA0021112005F07EF9C9
:104F0000112005F05FFAFEF77BF806F071FD032231
:104F100046494748FFF742FF2D24030004221C7036
:104F200044490130FFF73AFF30230470424D434CAF
:104F3000437083702E3B062220004149EB87FEF729
:104F400021FA062813D0200006F0A2FC022809D07E
:104F50000321200006F0F4FB8D23E3706E3B2371E8
:104F600019336371062220003549FEF745F9354BA8
:104F70001B68FC335C64FFF761FF0020FFF78AFFCA
:104F8000314C324A0121324B1278207801F0B4FFC3
:104F9000304A314B12780021207801F0ADFF012218
:104FA0002E4B1A702E4B5B78552B31D12D4B3B324B
:104FB0005A722D4B2D4AAB81EA812B826A822021C5
:104FC000307806F025FC0120404205F0CDFB0120A1
:104FD000404205F069FCFFF781F9FEF745FF00F05C
:104FE0009FFC01204042FFF70BF8012006F0F8FA81
:104FF000F72001F03DF90121307806F0D1FA307840
:1050000002F014F91A4806F043FBFEF745FE70BDA6
:105010006422184B5B7953431A000A32CBE7C0462F
:10502000B064FF1F554D0011694D00111446FF1F5C
:105030004C64FF1F6C64FF1F9E45FF1F6509FF1F27
:10504000ADAC00003067FF1FDA66FF1F0045FF1F91
:10505000E144FF1FAE66FF1F8F66FF1F8066FF1FC4
:105060009064FF1F8464FF1FC4090000CE09000084
:10507000B264FF1F9464FF1FF8B50A0020230D00DF
:105080001A40194251D0534B1B78002B3CD0FFF7EC
:1050900027FB514B514C524E99686268737A8A1AB9
:1050A000DB039A4202D36160FEF7F6FD327A217A81
:1050B000531EDBB299422AD1FFF7C8F9637A002B5D
:1050C0001FD0013BDBB26372002B1AD1454B5B78DA
:1050D000552B01D106F004FCE37A002B0CD0002301
:1050E000414A424FE3721388380001331380FEF7C0
:1050F000D7FE390006F0B4F9642370795843FFF7FE
:10510000B7FD237A0133237220206840F8BD914215
:10511000D4D300232372FFF7C3F9344F3800FEF7CE
:10512000BFFE390006F09CF9C8E70BB2002B0ADA83
:105130002F4B187806F02CFC002801D006F0E8F977
:1051400080200002E1E70224214206D0234B012007
:105150001A72FFF79FFE2000D7E70B071BD5FFF75A
:10516000BFFA1D4B1D491E4C98684A68637A821A23
:10517000DB039A4202D34860FEF78EFDFFF790F9F9
:10518000FFF764F900F0E6FB2368DB0701D5FFF7C2
:105190002FF80820B9E71024214206D00D4B1B78C8
:1051A000002BD8D1FEF774FED5E70124214209D0A7
:1051B000104800F06DF806F0B3F92100112005F059
:1051C0001DF8C8E704240800204021429ED0FEF7C5
:1051D00033FFC0E7B266FF1FA064FF1F8464FF1F98
:1051E0009464FF1F9064FF1F7864FF1FE144FF1F5A
:1051F000B064FF1FC444FF1FF0B51B4B1B4F1B883F
:105200003A8804001A4E1B4D85B09A420DD8328858
:105210009A420AD3184B1A882B889A4205D1174A0A
:10522000174B12881B889A421BD0052001F076F894
:105230003B8802AA13803388019053802B88114D3C
:1052400093800F4B02A91B88D3800F4B2A781888B4
:1052500002F092FD0D4B08212878019A1C7006F08F
:105260006FFB05B0F0BDC0467E66FF1FD644FF1F32
:10527000D444FF1FD244FF1F7C66FF1F7A66FF1FC6
:10528000D044FF1FDA66FF1FD844FF1F7866FF1F58
:1052900013B50C4B1C78002C11D1002801D00A4BFF
:1052A00018600A4A0A4B11780A4A10780A4A019291
:1052B0000A4A0092002205F003F9200016BD1124CD
:1052C000FBE7C046D966FF1F7466FF1FD866FF1F45
:1052D000C866FF1FDA66FF1FB466FF1FB866FF1FB0
:1052E00010B5064B12201B78052B06D1044B132258
:1052F0001988044B187801F0EDF910BDD966FF1F2D
:10530000D844FF1FDA66FF1F10B500240122114B9D
:1053100052421870104B1C70104B1A8001F086FF1F
:1053200004220F4B21001A700E480C3206F0A8F927
:10533000102221000C4806F0A3F907220B4B1C6039
:105340000B4B1C700B4B1C700B4B1A700B4B1C70D7
:1053500010BDC046DA66FF1FD966FF1FD844FF1F85
:10536000D866FF1FC866FF1FB866FF1FB466FF1F21
:105370008E66FF1F8D66FF1FDA44FF1F8C66FF1FBE
:10538000F8B5174C0600257806A814240078052DDA
:1053900023D1B41F134FA5B21824BD421DD88D1FB1
:1053A000ADB2BD4219D8FA256D00AA4215D21D0032
:1053B0000D4F0A3DADB2BD420FD80C4C26800C4CAF
:1053C00021800C4900240A800B4A1380FFF714FF48
:1053D0000A4B0421187806F03BF92000F8BDC046BE
:1053E000D966FF1F790C0000750C0000D644FF1F22
:1053F000D444FF1FD244FF1FD044FF1FDA66FF1FB3
:10540000F0B50BB20D0089B0002B00DB70E1A44EAB
:10541000307806F0BDFA041E50D00378A22B00D1DC
:1054200022E1D02B1AD0912B45D143780E2B42D1BB
:105430009C4B82889A423ED19B4A83681278052A07
:1054400039D1032018567F2835D0984B1B68002B84
:1054500031D05B68002B2ED098472CE0807807284D
:1054600029D806F095F80428183F3F74A8D8637827
:10547000002B0CD101218C4B19708D4B1A78002A0E
:105480005BD08C4B307801F037FD002855D00722D7
:10549000854B1A7051E061780029F8D1E378002B30
:1054A00011D0854A854B1278307801F025FD607067
:1054B0006378002BEBD1200006F02AF88020000250
:1054C000684009B0F0BD784B1B78022BF3D0012166
:1054D000307806F0B5F80028EAD10121307806F0DE
:1054E0005FF8E5E76378002BD1D16F4F032807D130
:1054F0003B78052B02D101333B701EE00223FBE712
:105500006F4B1A886F4B0293002A0BD01B78002B2D
:1055100003D00121307806F013FA3B78062B04D132
:10552000013BE9E7029B1A70F7E7042B41D1012107
:10553000029B3078197006F033F85C4B1B68002B27
:10554000B9D01B68002BB6D0574A107884E763782F
:10555000554F002B27D10622211D5B4806F030F85D
:1055600062895A4B5A491A80A2895A4B1A80E38998
:105570000B800521397058490A80584A1380228AC5
:10558000574B1A80574B1B78012B09D11F2000F075
:10559000C5FEFA22920042430421307806F0D0F989
:1055A0000022484B75E7312B00D070E70022454BB5
:1055B0001A700323A0E706220021434806F060F892
:1055C0000023454A04211380444A30781380444A1A
:1055D000138006F03DF80821307806F039F8A379F9
:1055E000083B5A425341304A03331370304B1B7807
:1055F000002B06D0334B30781A78002A06D001F001
:10560000B9FC0122314B52421A8096E701211970F0
:1056100005F0C6FFF5E70821307806F019F8637841
:10562000002B00D047E72C4B2D4F0293E388029AC2
:1056300004211380294B307803932389039A138024
:1056400063893B8005F0FCFF002800D033E7264B40
:105650001B68002B00D12EE7039902983A8809882D
:1056600000881B68984726E74379132B00D022E770
:105670000389012B0AD11D4B1B78022B06D108216F
:10568000307805F0E5FFFFF72BFE14E7052000F06A
:1056900045FE08210200307806F052F90BE7C046BB
:1056A000DA66FF1F05140000D966FF1F7466FF1F2E
:1056B0000045FF1FE144FF1FAE66FF1F8F66FF1FFF
:1056C000B066FF1FB266FF1F8166FF1FD844FF1F31
:1056D0008866FF1F8A66FF1F7E66FF1F7C66FF1FAE
:1056E0007A66FF1F8066FF1F7066FF1F7866FF1FC8
:1056F0008020C001014200D0E2E6CB0731D5324B19
:105700001B78002B1DD0314E05AC3378052B1AD1F8
:10571000023B23702E4B21001B7823722D4B1B78EC
:1057200063722D4B187801F08BFB002809D00720FD
:105730002A4B30701B68002B03D01B68002B00D055
:1057400098470120BCE60E20254B06221B782549F0
:105750002370254B1B78637002ABC01805F030FF37
:10576000D8E7022308001840194209D0174B1B78CC
:10577000052B03D11D4B188805F042FE02209FE641
:105780000424214203D0FFF737FD200098E60823C8
:1057900008001840194200D193E6154B1C78012CE3
:1057A00003D0022C0DD008208AE6124B124A13496E
:1057B00013481B881288098800880094FFF7E0FDD1
:1057C000F1E7FFF78DFDEEE7B266FF1FD966FF1F19
:1057D000DA44FF1F8C66FF1FDA66FF1F7466FF1F27
:1057E0008E66FF1FDB44FF1F8D66FF1FD844FF1F1F
:1057F0007866FF1FD044FF1FD244FF1FD444FF1F11
:10580000D644FF1F10B502A804880B20002C10D12D
:10581000496808784978090201430C48814209D156
:10582000022119800A4B59881170DB7800205BB285
:10583000537010BD074C0A20A142FAD102211980F1
:10584000034B998811705B79F0E7C0466E2A00001F
:105850007864FF1F6F2A0000F7B5150008AA1688A4
:105860004A680F4F14785278120222430A24BA422F
:1058700014D10122DBB2019200962A0005F026FD28
:10588000041E0BD1074B1B68002B07D068782A78C1
:105890000002104342425041013098472000FEBDB3
:1058A00002290000EC66FF1F30B5012503790400D2
:1058B000BFB02B4227D01549408805F073F8284225
:1058C0000DD06A46124B69465B8D138002235380CC
:1058D000104B5B8893806088002202F043F90E49E8
:1058E000608805F05FF8C0070DD56A460B4B694626
:1058F0001B88138002235380064B9B88938060880B
:10590000002202F02FF93FB030BDC046E466FF1F11
:105910000445FF1F7864FF1FDC66FF1F5E45FF1F05
:1059200010B5074C0749200004F0F2FF200006499B
:1059300004F0EEFF0721054A054804F0ABFF10BD57
:10594000FFFF0000E466FF1FDC66FF1FF4BB0011D1
:105950000445FF1F10B5024802F086FF10BDC04687
:10596000A95800110200F0B501270A480A4E511843
:105970008B1A002B00DCF0BD082415784308684022
:1059800038404000805B013C58406D08002CF5D148
:105990000132EDE7FFFF00000EBC0011F0B500255D
:1059A0000F269D4200DBF0BD4C5D070944403440AA
:1059B000A400A05801357840F3E70000F0B589B0A5
:1059C0006A460D000B000F27110010351C780133BB
:1059D000260024093E40167054700232AB42F5D1C5
:1059E0002023024AFFF7DAFF09B0F0BD14BC001112
:1059F000F0B54E780B7889B036020C001700019094
:105A00001E43012A61D9954B9E4200D877E00133AD
:105A10009E421CD1062A17D1CA788B7812021A43EB
:105A20000B791B0413434A7912061A438C4B5A61B3
:105A300000221A705A808B4A5A608B4A9A608B4AAD
:105A4000DA60002009B0F0BD88225205EEE7884BED
:105A50009E423CD182498B78002B00D0F6E00C2A84
:105A600031D10F22A3789343E278120213432279B3
:105A7000120413436279120613434B60E279A07952
:105A800012020243207A00041043627A1206024393
:105A9000CA60E27AA07A1202024376484A818342BF
:105AA00008D804236E49142201980B7005F088FD74
:105AB0001420C7E71201D21889235B059A42F0D857
:105AC00001238B70BDE7022AFAD00523EAE76A4A70
:105AD00001239642E6D1FFF703FC052F0CD9E378AA
:105AE000A2781B021343227912041A4363791B061E
:105AF0001343624A0393136005F0F2FEA1E7584D89
:105B00002B78002B9DD1AB78002B00D1A0E02B8906
:105B100001339BB20093B34200D091E0132AD4D951
:105B2000CF7C8B7C3F02122120001F43FFF71AFF1E
:105B3000874200D08EE0002E3DD1E378A2781B0290
:105B400013432279E96812041A4363791B0613434D
:105B500003930A228B4212D1FF23A370E3702371B7
:105B600063716B89002B09D1E37B227C1B02120439
:105B70001343A27B13431B0901336B8100226B8902
:105B8000002B8ED0002A67D1686837013818000BC7
:105B90006B6900030390984205D9686105F080FCA9
:105BA000EB780133EB7068681022A11C381805F0FF
:105BB0005FFD2E8145E76F89009A7B1E9BB2934261
:105BC0003AD1E278A37812021A43237905A81B047C
:105BD000134362796C6812061A43EB6800920392D1
:105BE000211D0C22049305F0EBFC0120260004A9E2
:105BF00040421036FFF7E2FE013F012F17D1009A15
:105C00000B232861824200D04CE704221C4920006B
:105C100005F02EFD042203A9686805F0A9FCE968D7
:105C2000039AFF23914200D13CE7F73B3AE731006A
:105C3000FFF7C4FE1036DFE70923B742A4D831E7E7
:105C4000009BB34200D9FCE607232BE7022329E798
:105C5000032327E7062325E70A2323E7FFFE0000A7
:105C60007845FF1F00000111FFFF00005048593622
:105C700001FF0000FFFF001102FF000034F00040B0
:105C80008445FF1F10B5034C0B000122210000F0DA
:105C90006BFA10BD455E00110B8870B506000D0053
:105CA0000224162B11D92B000322094900F05CFABB
:105CB000041E0AD1074B2A881B88191C934200D95D
:105CC000111C300089B200F0EFFA200070BDC04610
:105CD000715E00114A67FF1F10B54A780400013A4F
:105CE0000B000220012A07D80A78002A04D00522D6
:105CF0002000024900F038FA10BDC0469F5E001136
:105D00000A7810B50B0004000220002A04D00722F4
:105D10002000024900F028FA10BDC0464B5F001178
:105D20000A7810B50B0004000220002A04D00922D2
:105D30002000024900F018FA10BDC046B15F001102
:105D400010B5034C0B000B22210000F00DFA10BD22
:105D5000E15F001110B5034C0B000D22210000F093
:105D600003FA10BD5360001110B5034C0B000F2255
:105D7000210000F0F9F910BDAD6000110A7810B5EE
:105D80000B0004000220002A04D011222000024946
:105D900000F0EAF910BDC046BD600011002310B547
:105DA0001322190000F0E0F910BD000010B5034CFB
:105DB0000B001722210000F0D7F910BD0F61001170
:105DC000002310B51922190000F0CEF910BD000013
:105DD00010B5034C0B001B22210000F0C5F910BDCB
:105DE00049610011F7B584890D0006000121002CDE
:105DF00022D000238268D3561778002B1EDA0C2C91
:105E00001AD90C3CA4B2131940880093230002F065
:105E100086FE431E984101307B06DB0F6B703F23EB
:105E2000013C1F40A4B22870AF70AC80002C07D09A
:105E3000B3680133AB6000210800FEBD0020EBE732
:105E4000AC60F8E70B7803704B8843704B881B0AF3
:105E500083700B79C370042070470420022B06D195
:105E60000020537811781B02009A0B43138070476F
:105E70000B8803700B881B0A4370022070470420B4
:105E8000009983420AD1537810781B0203430B8098
:105E9000D37890781B02034300204B807047F8B5FD
:105EA0000D004B7801240021461C03702B788B4297
:105EB00001D82000F8BD6B78B01C4F1C012B10D10D
:105EC000890069184B88022233704B88B9001B0A7D
:105ED0007370691805F0BCFA04360434A4B2F9B240
:105EE000E4E7122359436B185A88043132705B88F7
:105EF00010221B0A7370691805F0AAFA12361234C0
:105F0000ECE770B5049D14001E00052B01D8042099
:105F100070BD637812781B0213432B80E378A2785C
:105F20001B02134302226B802A71211D681D063E4D
:105F300005F08EFAB2B22A81F02AE8D82800A11D15
:105F40000A3005F085FA0020E2E7002310B50A7850
:105F50009A4201D8900010BD9A008A1854880133E3
:105F600004705488DBB2240A447094888470928848
:105F7000120AC2700430EAE710B51100029C062B29
:105F800004D004201022142B01D010BD0222227153
:105F90004B7808781B0203432380CB7888781B0258
:105FA000034363800431601D05F052FA0020ECE7E2
:105FB00010B50C788B7804315C43E4B20370220096
:105FC000013005F045FA601C10BD0420022B06D1FB
:105FD0000020537811781B02009A0B4313807047FE
:105FE00010B50C000A88023105F032FA208810BD85
:105FF00070B504000D0004981100012B01D8042095
:1060000070BD167852781202324302800200F832D4
:1060100055701470E825002C00D10C35023B9AB263
:106020004280AA42EBD80231043005F011FA002078
:10603000E6E70420009983420AD1537810781B02C6
:1060400003430B80D37890781B02034300204B80DE
:10605000704710B50C000A88023105F0F9F9208864
:1060600010BD000070B501211E000420049C0E40EC
:106070000B4218D1CB40DDB28D4214D90A49DBB2B4
:10608000098899420FD32300F6331D70330058005E
:1060900011184978165C0902314301332152D9B2F3
:1060A0008D42F4D8002070BD9845FF1F10B50C003C
:1060B0000A88023105F0CCF9208810BD10B50C78A3
:1060C0008B7804315C43E4B203702200013005F0A8
:1060D000BFF9601C10BD10B511000298032B01D848
:1060E000042010BD14785278043B1202224302802F
:1060F000CA788C781202224342809AB28280F22AB5
:10610000EED80431063005F0A3F90020E9E710B518
:106110000C000B8803700B881B0A43704B8883703C
:106120004B881B0AC3708A880430063105F090F949
:10613000A088043080B210BD0420012B03D10020C0
:106140001378009A1370704710B50C000B88037019
:106150000B881B0A43704A880230043105F078F935
:106160006088023080B210BDF0B589B003931E4B39
:10617000029242000700D05A019102F020F8132544
:10618000061E2DD0029B01240370019B002B04D01E
:10619000001903999847001984B26B461B7A5BB2C9
:1061A000002B0FDA1021380002F01CFB1925002803
:1061B00013D130003219E1B202F066FC051E0CD199
:1061C0000C34A4B2042304AA380005A993800696CF
:1061D000948101F0AFFD051E02D0300005F0A8F952
:1061E000280009B0F0BDC0464867FF1F70B5050024
:1061F0000C0000280CD00020814209D01022200081
:10620000044905F025F901202B7823736B7863731B
:1062100070BDC04654BC0011F0B506000D0017005B
:106220001C0085B002291BD00020102907D1022BA9
:1062300007D0102B03D115E00020102C08D005B09A
:10624000F0BD69463800FFF7D1FF2A0069460BE030
:1062500069463000FFF7CAFF22006946380004E0B3
:10626000022BE9D12A003900300005F0E9FAE6E70F
:10627000031CF72800D9F723032008499AB2013AF2
:106280000B80D317034006499B189B100B80D30F3C
:1062900004499B185B100B807047C0469C45FF1F4C
:1062A0009A45FF1F9845FF1F034B1B888B4202D363
:1062B000024B4000C15270479C45FF1F4867FF1FBB
:1062C000014B4000185A70474867FF1F1722014BC7
:1062D0001A8070474867FF1F70B505000E2005F053
:1062E0001FFA041E13D0D0230370002306228370EC
:1062F00007494570033005F0ABF8064B2100DA8AF8
:1063000062811B7E2373044B187805F0F1FA70BD8F
:106310006467FF1F5467FF1FEC45FF1F262803D843
:10632000024B4000C05A70470148FCE79E45FF1FE2
:10633000FFFF000070B506000C00094D1C22002173
:10634000280005F09DF9074B1E70074B1C7005F0E7
:10635000EFF90123002801D0002312202B7070BD1B
:106360005467FF1FEC45FF1F7567FF1F70B50500E1
:106370000D4C0800E260A16010220021656005F06C
:1063800097FA012803D11021A06802F058FD1022CD
:106390000021280005F08CFA012803D11021606843
:1063A00002F04DFD70BDC0465467FF1F70B5041E5E
:1063B00005D1002903D006220D4805F049F80D4B00
:1063C0001D78012D11D1002C05D102221A7005F083
:1063D0007FF8280070BD00221A70074B1B78FF2B36
:1063E000F7D02000FFF778FFF3E70025F1E7C0467C
:1063F0006467FF1F5467FF1FEC45FF1F030010B5C4
:10640000002801D1002010BD00780B4A002803D1DC
:106410005988D1821B7913761378022BF2D100238D
:10642000984200D103331370044B1B78FF2B01D02B
:10643000FFF752FF0120E6E75467FF1FEC45FF1FFF
:10644000002911D000280CD04B79012803D140221B
:106450005242134303E03F221340032802D001209D
:106460004B7170474022F4E70800FAE770B5094D18
:106470000100287800280BD0074C0622200004F0E9
:10648000E7FF21002878FFF7DBFF200005F060F927
:1064900070BDC0467467FF1F4E67FF1F00290AD0FA
:1064A000012808D13F224B799343C02B03D0403BB6
:1064B0005A425341981C704770B5174D06002B780F
:1064C000FF2B15D00A2005F02BF9041E10D0D02385
:1064D0000370C83B8370114B11491B784670C37021
:1064E0000622043004F0B4FF2100287805F000FAF9
:1064F0000C4B1B78012B0DD10B4B1B68002B03D0D1
:106500009B68002B00D09847084B04211878084A54
:1065100005F086F870BDC046EC45FF1F7467FF1F8D
:106520004E67FF1F7067FF1F9C67FF1FA067FF1F5D
:1065300060EA0000014B98687047C0465467FF1F2F
:10654000014BDB68186870475467FF1F074B10B595
:10655000DA68136801331360054B1878FF2803D0FD
:106560008021C90105F01CF810BDC0465467FF1F0B
:10657000EC45FF1FF7B50E0002F0C8F8051E1CD051
:106580000E4B06621F78002F00D10778AB791020E0
:10659000019305F0C5F8041E0FD0D0230380C73B3C
:1065A0008370019BE91DC3700622043004F050FF84
:1065B00021003800E66005F09BF9F7BDEA45FF1FB2
:1065C000014B18787047C0467467FF1F054B0028C1
:1065D00005D1054B1A78054B002A00D1014B180054
:1065E0007047C0466467FF1F7467FF1F4E67FF1F39
:1065F000014B58687047C0465467FF1F024B18682C
:10660000431E9841C0B270477867FF1F421E0300C7
:106610000120152A03D9FF3B5A425341D8B2704793
:10662000F0B51C0000230E0085B0039002920B70A1
:10663000029A934201D3002019E0E55C5A1CD2B2C1
:10664000002DF8D0029851198142F4DC0233DFB2F8
:10665000A35C18000193FFF7D9FF002807D0013D84
:10666000019A0399EBB233708A4202D1E01905B066
:10667000F0BDDB19DBB2DBE710B50C0002F09EF8D1
:1066800003001220002B03D02100588805F048F9A0
:1066900010BD000070B50E4D84006359002B15D05D
:1066A000186A002801D004F0C3FF2B59586A00284B
:1066B00001D004F0BDFF2B59986A002801D004F0E6
:1066C000B7FF285904F0B4FF00232B5170BDC0461A
:1066D0008467FF1F1C4B70B504000E001500994223
:1066E0000AD11A4B1B68002B01D1122070BD1B6808
:1066F000002BFAD09847F9E7154B994215D1134B67
:106700001B68002B0AD01B68002B07D09847002875
:1067100004D1104B1C70104B1D70E7E729002000BE
:10672000FFF7AAFF0028E1D1F3E7080001F0EEFF30
:106730000028DAD003780320A342D7D12900300003
:1067400005F0EEF8D2E7C046FEFF00008067FF1FAD
:10675000FFFF00007D67FF1F7C67FF1FF7B5040088
:10676000808801F0D3FF0025A84203D00578A088D7
:1067700002F008F81C4E3378002B1FD0AB421DD11D
:106780001A4B28001978FFF777FF002818D000234C
:106790003370A3790820A778A688019304F0C0FF7E
:1067A000011E0DD0D0230370CA3B8370019B47703C
:1067B00086808371280005F09BF801E0002DE8D168
:1067C000A0880B4B8200D358002B01D0FFF762FF4B
:1067D0001721A088FFF768FDA08801F027FDA08899
:1067E00001F0FEFDF7BDC0467D67FF1F7C67FF1F00
:1067F0008467FF1FF0B587B01D000CAB1B88070036
:1068000001930DAB1B88142002930EAB1B8816005E
:1068100003930FAB1B880091049310AB1B88059367
:1068200004F07EFF041E1AD0D0230370CB3B4770C8
:106830008370C670062229000430002D11D004F0A8
:1068400007FE019B21006381029B0098A381039BAB
:10685000E381049B2382059BA37405F049F807B0EC
:10686000F0BD04F00DFFECE7F7B5009308AB1B8813
:1068700007000C200D001600019304F051FF041EC8
:1068800013D0280001F042FF00280FD00078D02359
:106890002370C93BA370009B21002381019B67707B
:1068A000A580E680638105F023F8F7BD014B1878D9
:1068B000EDE7C046EC45FF1F13B50400648903896A
:1068C000C2888188C0780094FFF7CEFF13BD000016
:1068D00010B5044C2068002803D004F0A9FE002362
:1068E000236010BD8867FF1FA122F0B58188920048
:1068F0004A43384B384F1B6804009B189D22920076
:106900009B18827989B01A603B68002B5FD01D7894
:10691000324B1B68002B04D05B68002B01D0002099
:106920009847260008363100E079FFF7B7FD237D50
:10693000E0710200E0780493638A29000393238ABC
:106940000293E3890193A38800933300FFF752FF7A
:10695000E378002B0BD1E289A379A18802920196FA
:10696000E27928000092012201F0DAFEE0703B6833
:10697000002B20D0FFF7ACFF194D287800281AD043
:10698000184B1978FFF778FE002814D02B78E6789A
:1069900008200793A78804F0C3FE011E09D0D02366
:1069A0000370CA3B4670837087808671079804F035
:1069B0009FFF00232B701721A088FFF775FCA0888C
:1069C00001F034FCA08801F00BFD09B0F0BD064BCE
:1069D0009DE7C0463409FF1F8867FF1F9C67FF1FA4
:1069E0007D67FF1F7C67FF1FEC45FF1FF8B50700A1
:1069F00008000E0001F08AFE041E18D02620FFF7C2
:106A00008DFC051E00D12578062004F089FE041EA9
:106A10000DD00021062204F033FED0232370C23BA8
:106A200021006770A370A680E8B204F061FFF8BD92
:106A3000F0B585B001930AAB1B78070002930BAB4E
:106A40001B7808000D000092039301F05FFE061E04
:106A500022D0102004F064FE041E1DD0102200215C
:106A600004F00EFE2620FFF759FC002800D13078F4
:106A7000D0232370C13BA370009B21002372019B94
:106A800067706372029BA580A372039BC0B2E3721E
:106A90000C9BE36004F02CFF05B0F0BDF7B50D00D2
:106AA000019001F033FE071E20D00E2004F038FEC6
:106AB000041E1BD02620FFF731FC061E00D13E78B5
:106AC000D0232380C53B0622A370F91DE01C04F0EF
:106AD000BFFC019B2A0063810123DD401A401D4059
:106AE000210022736573F0B204F002FFF7BD0000CD
:106AF000F0B585B0029010000D0017000A9E0393B8
:106B000001F004FE041E31D0029B002B2ED1039B0A
:106B100002795B0724D5122313430422002E08D1E7
:106B20000B99002905D10C99002902D10D99002952
:106B30001AD01A430D9B2271002B00D0C9E0002E01
:106B400000D1CFE0002D00D0CCE0606A002801D059
:106B500004F06EFD1C21300004F0DAFD606205E0F7
:106B600002239A430E33D7E793432371654BBA0050
:106B7000D458002C00D1AAE0002E10D0236A002B9C
:106B800003D11C2004F054FE20625E4BBA00D3589F
:106B9000186A002803D01C22310004F059FC0C9B19
:106BA000002B12D0574CBB001D596B6A002B03D130
:106BB000162004F03DFE6862BB00E358586A0028C6
:106BC00003D016220C9904F043FC0D9B002B11D02E
:106BD0004C4DBC006659B36A002B03D1142004F05D
:106BE00027FEB0622B59986A002803D014220D9911
:106BF00004F02EFC380001F089FD051E67D0414BE2
:106C0000BA00D358002B62D01A6A3420002A00D16F
:106C10001C389A6A002A01D0143080B20B9A002ADC
:106C200001D01C3080B25B6A002B01D0163080B2DC
:106C300004F076FD041E4AD01822002104F020FD45
:106C40002620FFF76BFB0190002801D12B780193E0
:106C5000D0232370029B200063700A23294EA37067
:106C6000039BBD00A371AB59A780196A1830002996
:106C700005D01C22A06004F0EBFB200034307359D7
:106C8000996A002907D0030014221433E0600293AC
:106C900004F0DEFB02980B9B002B08D003001C22A3
:106CA0001C330B992061029304F0D2FB02987359B4
:106CB000596A002903D01622606104F0C9FB6B46B3
:106CC0002100187904F014FE3800FFF7E3FC05B04A
:106CD000F0BD10220D9B0D991B69A018236204F0D2
:106CE000B7FB2CE70B9B002B00D13FE7012D00D019
:106CF0003CE7606A002801D004F09AFC1C210B9844
:106D00002AE7C0468467FF1F10B5044C206800289E
:106D100003D004F08DFC0023236010BD7867FF1FB3
:106D20000B4B07B51A68002A01D100200EBD694639
:106D3000531C012012780731FFF772FC0028F4D0B1
:106D400002780123100018401A42EED0EEE7C04648
:106D50009467FF1FF0B51F4F01203B6887B0002BE1
:106D600025D09B78059300F0B3FB002821D00A20A2
:106D7000FFF7D4FA04000B20FFF7D0FA164B0500FA
:106D80001E78731E9E413B68F6B2191DD878FFF736
:106D900057FB3B682900DA7A043303929A7901930E
:106DA0000292009033002000059A04F041FB07B0E6
:106DB000F0BDFFF7B5FF002805D00620FFF7AEFABB
:106DC00004000720D8E70820FFF7A8FA04000920EC
:106DD000D2E7C0467867FF1F7467FF1F70B50A4E81
:106DE000040033780D00FF2B0DD0042004F098FC34
:106DF000011E08D0D0230370CE3B45708370C47051
:106E0000307804F075FD70BDFC45FF1F70B50400BF
:106E100006200D0004F084FC011E0AD0D02303706C
:106E2000CD3B8370054B44701B688580187804F057
:106E30005FFD002C01D0FFF767FF70BD7867FF1F73
:106E4000F8B5264F06003B680D001124002B05D134
:106E50000522234B1B78134202D112242000F8BDD7
:106E6000204A10241268002AF8D01278002AF5D09F
:106E7000DB0719D52B789A1E012A1AD80C2004F0AA
:106E8000D7FC132438600028E8D000230A2243707E
:106E900029000670023004F0DBFAFFF75BFF041EE6
:106EA0000AD0FFF731FFD9E700F012FB0028E1D14B
:106EB000E4E7002BE2D0D0E70B4B1B78032BCDD1BE
:106EC0001D20FFF72BFA094B18800028C6D0084B6D
:106ED00004211878074A04F0A3FBBFE77867FF1F77
:106EE0007567FF1F9467FF1F7467FF1F7267FF1F9F
:106EF000A067FF1F60EA0000F7B50193194B14006B
:106F00001A78052306000F0012201A4221D0012909
:106F100020D1154B1D68002D1BD002201F2C18D826
:106F2000002C02D0019B002B13D0104B1F221E708F
:106F30006E1C0021300004F0A3FB019922003000F8
:106F400004F086FA310020002C70002F06D004F0E7
:106F5000D7FAFEBD064B12201D68DCE704F0B8FC32
:106F6000F7E7C0467567FF1F9467FF1FFC45FF1FCB
:106F70009067FF1FF8B50F4E12243368002B17D00F
:106F80001B780F3C834213D100250B4F0221387828
:106F900004F05EFB094B042138781D8004F058FB97
:106FA000074B28001D8033685C7004F089FB0400E7
:106FB0002000F8BD7867FF1FA067FF1F8C67FF1FC9
:106FC0007267FF1F70B5012823D11B4C2388002B4B
:106FD00003D01A4A1578002D07D0194B1B68002BD7
:106FE00002D01878FFF7C6FF70BD3B2B02D93C3B9F
:106FF0002380F9E7134E0221307804F029FBFA22AE
:107000002388920002215A43307804F099FC2580AD
:10701000EAE70B4B1B68002BE6D00B4B1B785B079A
:10702000E2D5084B0221187804F012FB0022024B33
:107030001A80FFF769FED7E78C67FF1F7067FF1F95
:107040007867FF1FA067FF1F7567FF1FF8B51E4D0C
:107050002868002803D004F0EBFA00232B601B4EB5
:107060003068002803D004F0E3FA00233360184F9F
:1070700005243B7818002040234221D0154800F019
:107080002BFA3B78234213D0202004F0D1FB286058
:10709000002813D02022002104F0F2FA202004F06E
:1070A000C7FB041E306005D02022002104F0E8FA5E
:1070B000002004E0286804F0BBFA2C601320F8BD1F
:1070C00000F00AFAF4E7C0469467FF1F9067FF1FBD
:1070D0007567FF1FF045FF1F10B50A4C23681A1E85
:1070E0000ED0002808D10130587004F0E9FA0028C9
:1070F00005D02368002B02D00021FFF787FE012274
:10710000100010BD7867FF1FF7B5274E05003368E4
:107110000191181E21D05C78244F012C30D1FFF74B
:10712000FFFD002825D02000FFF7F8F804004128D3
:1071300014D91F4B022118781E4A04F071FA1E4B15
:107140003C3C1C80022233685A703B78002B14D1DF
:1071500028000199FFF75AFE0120FEBDFA22920095
:107160004243002AEED0124B0221187804F0E8FBCB
:10717000E8E7FFF7D3F80200F3E700233B70EBE703
:107180003B78002BE8D1032004F0CAFA011E08D096
:10719000D0230370CC3B457083703368187804F0BB
:1071A000A7FBFFF7B1FDD7E77867FF1F7067FF1FE9
:1071B000A067FF1F60EA00008C67FF1F10B517492A
:1071C000838802008B4220D011D815498B4217D0FA
:1071D000144900205B1899B2012907D892681178E8
:1071E0005A425341D8B2FFF7F9FD012010BD0E4AB3
:1071F00000209B1807229BB29A424041C0B2F5E79B
:1072000083681878FFF768FFF0E7836899785A7801
:10721000090218781143FFF777FFE7E70A2000001B
:1072200006200000F8DFFFFFAFDFFFFF014B187003
:107230007047C046FD45FF1F10B5064C207001F099
:1072400041FA207804F0F4FB0521207800F062FD7B
:1072500010BDC046A067FF1F0BB273B50D00002B19
:1072600000DBC4E0884B187804F092FB041E0ED0BB
:107270000378912B0FD0A22B00D1A1E0834B18787B
:10728000FF2852D0210004F033FB00284DD180208C
:107290000002684076BD43780F2B76D013D8052BBB
:1072A00070D00E2BEAD18088794B98422BD8794B3D
:1072B00098421BD8784B9842E0D1A3681878591CA3
:1072C000FFF774F838E03E2BD8D18378032B74D0C5
:1072D0006CD8012B6ED0022BD0D1704B1B68002BC9
:1072E00023D05B68002B20D098471EE06C4BC01861
:1072F0000C28C3D804F0C4FA1DC2C2150BC20B0B74
:107300000B3223C23C00674BC0180728B6D8664B27
:107310001B68002B09D01B68002B06D02000984763
:107320000AE0A3681878FFF7C7F8200004F0F0F827
:10733000ADE7A068FFF762F800289FD0F5E7A368E3
:107340001B78002BF1D0554B1B68002BEDD01B6830
:10735000002BEAD0210055489847EDE74F4B1B68BA
:10736000002BE2D01B68002BDFD021005048F3E750
:10737000504B1B68002BD8D05B68002BD5D0210068
:107380004348E9E7FFF7EAF9CFE780884A4B98429C
:1073900003D04A4B984200D070E7464B1B68002B45
:1073A000C3D05B68002BC0D02100D5E7153B012B73
:1073B000BBD963E7FFF798FAB7E7FFF77DFAB4E7C1
:1073C0003F4B1B78042B07D100236A4613800179B9
:1073D000408800F0C5FCA8E7364B1B68002BA4D002
:1073E0005B68002BA1D00100364898479DE7012437
:1073F00021420AD0294B1B68002B04D05B68002B6C
:1074000001D000209847012043E78B070AD5264B7F
:107410001B68002B04D05B68002B01D0200098472C
:10742000022036E70421280008400D4200D131E750
:10743000254E3388002B21D0013B9BB23380002B9B
:107440001AD1FFF7DBF800280AD0204B1C70164B2E
:107450001B68002B04D05B68002B01D020009847EC
:10746000FFF7C6F8694601F001FD6846FEF7FEFF2A
:107470001D20FEF753FF308004200AE7024B1878E6
:1074800004F0E6F8F8E7C046A067FF1FFD45FF1FC0
:107490000E20000001200000091000009867FF1F67
:1074A000FEDFFFFFAFDFFFFF9C67FF1F0C20000028
:1074B0000B2000008067FF1F0D200000132000003C
:1074C0007567FF1FFFFF00007267FF1F7067FF1FD8
:1074D00010B501F09BF910BD014B18607047C04614
:1074E0009C67FF1F0B880020162B01D81723042050
:1074F000014A13807047C0464A67FF1F002070474B
:10750000074A03001188814207D0918800209942E0
:1075100002D101308000101870470020FAE7C04601
:10752000A867FF1FF0B58F7806000D00C7B01E2FAB
:1075300015D1FFF7E5FF051E03D10024200047B059
:10754000F0BD00223B003100C078009200F0B2FB99
:107550000400A81C00F0D3FBFF23EB70EEE7264BE2
:10756000062403931B78FF2BE8D0182FE6D87B085E
:10757000224A013BDB0002929A589446002ADDD051
:10758000029AD3185B68002BD8D00878002802D163
:107590004B78012B02D10624122FCFD107AFAB8835
:1075A000697800976446AA68A047041EC6D1AB78E4
:1075B000029A5B08013BDB00D318390030005B689E
:1075C0009847041E0BD1AB78042BB6D0039A310038
:1075D00010782200009700F06DFB0400AEE76A7897
:1075E000002AABD1AA7805A93B88087130000A703F
:1075F0004B80FEF747FBA0E70046FF1F64BC00116D
:107600001D4B37B5050098420BD000290AD1FFF772
:1076100077FF002805D11948FFF772FF002800D036
:10762000058037BD01291AD1FFF76AFF041EF8D083
:1076300001235B420380A378FF2BF2D0FE2B07D0FF
:107640000023E0781422009329001E3300F032FB5F
:10765000A01C00F054FB01235B426380E1E7022998
:10766000DFD1013901F0BEF80028DAD12800FFF798
:1076700047FF041EDFD1D4E7FEFF0000FFFF00003C
:10768000022210B5074B52421A80074801325A8035
:107690009A80DA8000F07EFA044801F025F8002094
:1076A00010BDC046A867FF1F2575001101760011A7
:1076B0000388F7B50400002B02D102252800FEBD87
:1076C00042680221137825485268FEF7A5FD00287C
:1076D0002ED0234F01253A88002AEFD0802321881D
:1076E0005B0201259B1A9942E8DC0C2004F0A0F80B
:1076F000061E31D03B8822889C4600231800019545
:1077000061469DB2491989B2AA421BD8002801D00E
:1077100062443A8000233000082208C0210003F0B0
:1077200097FE104A1368002B13D100251660C5E799
:107730006268022113780C485268FEF76DFD00283C
:10774000C7D1BAE760681D01401941810133019832
:10775000D6E71A001B68E6E71325AFE7D2BC001195
:10776000FE45FF1FA467FF1FD0BC0011014B18701E
:107770007047C0460046FF1F14230A0010B51A4088
:10778000194204D00122102101F048F810BD4B0627
:10779000F9D4012088434000F8E710B514008B06A7
:1077A00004D50122102101F039F810BD08230A0088
:1077B0001A40194202D14BB2002B0FDA102101F00E
:1077C0002DF8002808D02300F9331B78002BECD0CB
:1077D000F8342378012BE8D10020E6E7032089075D
:1077E000FAD4E2E7F0B51F00184B85B01C68019091
:1077F00002910392002C27D1200005B0F0BDA568AE
:107800003301ED186B89019A934211D3029A934286
:107810000ED8002F04D10A9B002B10D12C00EBE7CF
:107820003B002978039A6868FEF7F6FC0028F2D13D
:107830000136B6B2A388B342E1D82468DAE7A36878
:107840000A9A5B891380E9E70026F3E7A467FF1F24
:1078500037B50C000A8849880123914217D3002AC2
:1078600015D0651D23792A0002210A48FEF7D4FCB1
:10787000102300280BD023796188208800242A0057
:107880000094FFF7AFFF0A23A04200D023001800A6
:107890003EBDC046D2BC001113B50A000888498815
:1078A000012388420BD8002809D00024137905321F
:1078B0000094FFF797FF0A23A04200D0230018008E
:1078C00016BD13B50A0008884988012388420BD8E1
:1078D000002809D00024137905320094FFF782FFB5
:1078E0000A23A04200D02300180016BDF0B58BB0CB
:1078F00003904A8808880E000123824255D300284D
:1079000053D00023012704AC237000227188130098
:107910000092FFF767FF051E3ED02078002835D182
:107920002B78022B18D167706A8983000130E31825
:1079300080005A8069680222201803F089FD2378AC
:107940000133DBB22370042B19D93B006889013065
:1079500080B2002BD9D01FE002236370122358435A
:107960006A89231804305A8069681022201803F0AD
:107970006FFD23780133DBB22370002BE5D10C4A75
:107980006B899B185A425341DBB2DFE76378012BC6
:10799000E4D12B78022BC7D022780A23002A04D006
:1079A00021000398FEF798F9002318000BB0F0BDF2
:1079B0000100FFFF0F4BF0B504001868002816D037
:1079C00083685D89A54207D88288AE18B44203DA7D
:1079D00012019A18934201D10068EFE71E005F89F7
:1079E0001036A74204D1002900D00D801800F0BD48
:1079F0003300EFE7A467FF1F70B505000C0008888F
:107A00000021FFF7D7FF03000120002B04D0220044
:107A10002800197AFFF7C1FE70BDF7B50C000025EC
:107A200001902300F6331B78AB4201D800200AE016
:107A30006B00E65A00213000E718FFF7BBFF002873
:107A400002D126800130FEBD017A0198FFF794FE35
:107A5000002802D03B882380F5E70135EDB2E0E74E
:107A600010B5040008880021FFF7A4FF03000120DF
:107A7000002B03D02000197AFFF77EFE10BD000016
:107A8000054B1B68002B01D1180004E09A6852894D
:107A90008242F6D198887047A467FF1FF0B50E2781
:107AA000002687B0039302ABFF183E8005001F4BF2
:107AB00040891400984207D02B78013000976A68FB
:107AC00080B2FFF78FFE060002212B7818486A6803
:107AD000FEF7A2FB00280FD06C892000FFF7D0FF33
:107AE000002802D0013C0419A4B2039B002B00D053
:107AF0001C80300007B0F0BD02212B780D486A6869
:107B0000FEF78AFB0028E7D102212B780A486A6831
:107B1000FEF782FB002807D0002EDED03B88A34270
:107B2000DBD17489013CDFE76C89DEE7FFFF0000F1
:107B3000D2BC0011D0BC0011CEBC001110B50C009D
:107B4000FFF7DEFC03000220002B0AD0002C00D03F
:107B500023609B781720FE2B03D00138FF2B00D128
:107B6000002010BD73B50D0001A904001600FFF739
:107B7000E5FF172805D0002E04D129002000FEF7CC
:107B800027F976BD01221021200000F047FE0028D1
:107B9000F3D0F6E7014B18607047C046B467FF1F8B
:107BA00037B56B469D1D010004000222280003F03A
:107BB00007FD2B88B02B0ED12379122B09D123007E
:107BC000FF339B78012B06D10121608800F0E0F89B
:107BD00001E01B2BF8D037BD10B5054B0421187000
:107BE00000F098F8FFF74CFDFEF770FB10BDC046A3
:107BF000B867FF1F0020F0B50BB20F0087B08342BB
:107C000034DA274B187803F0C3FE051E2BD0037817
:107C1000A02B25D103AE3100FEF7E4F8041E0BD1F2
:107C2000B378DB0724D51F4B06341B68002B03D029
:107C30003100688898470400A868002801D003F044
:107C400077FC002C08D1184A039B1340174A934233
:107C500006D0B3781B2B03D00121688800F098F878
:107C6000280003F055FC80200002784007B0F0BDEA
:107C70000F4B1B68002B10D0310068889847041EFA
:107C8000DAD07378002BD7D1B27801A90A704B8073
:107C90000C716888FDF7F6FFCEE70624F1E7C046D1
:107CA000B867FF1FB067FF1F00FFFF000001120051
:107CB000B467FF1FF7B50190822040000D00170048
:107CC0001E0003F02DFD04001320002C12D0B02361
:107CD00020002370089BFC226770658026710830A5
:107CE000002B08D0190003F0B3FB2100019803F02A
:107CF000FFFD0020FEBD089903F0C2FCF5E710B5BA
:107D0000041E06D00078FD2803D803F081FCFF2371
:107D1000237010BD0A1F93B210B504000220032B7C
:107D200005D882400020024BD1529B189C7010BD98
:107D3000D867FF1F0B8870B5043B04000D000220BC
:107D4000032B0BD80121200000F04CFD0300142070
:107D5000002B03D02900200000F0DEFB70BD0000E6
:107D600007B51300034A00920A00012100F02CFC21
:107D70000EBDC0469D7F001107B5019203220092FF
:107D8000024B0A00122100F049FC0EBD1B800011BD
:107D900007B56B4601AA11800449D88008780633DC
:107DA000012802D1190003F0ABFD07BDB967FF1F21
:107DB0000C4B10B518700023FF210B4A1380138160
:107DC00093819380094A5380137051729381937207
:107DD000D174D3821375517703F002FD00F0FCF9E2
:107DE00010BDC046E867FF1FD867FF1FBA67FF1FB7
:107DF000F0B58DB06B46002003910C229B5E834250
:107E000000DBB0E05D4B187803F0C2FD051E00D129
:107E1000A4E00378902B00D09DE006AF01004688D7
:107E2000380000F013FA79680400002900D19CE0C2
:107E30003B88052B6ED13B89032B1CD905AC200058
:107E400000F0A2F86288172A61D83989131D994277
:107E500031D17968237804310291D90738D5607817
:107E600000F08EF9071E06D0002303712378012B42
:107E700008D0132B23D0A868002800D178E003F0A5
:107E800057FB75E06288029909A800F0A6F80290F5
:107E9000380000F08BF909AA2378387A0192002281
:107EA00031000092029A00F012F9380000F064F9F3
:107EB000029B002BDFD0300000F080F9DBE7037875
:107EC000032BD8D16288029909A800F0D6F8DEE722
:107ED000122B13D1029909A800F0B5F8021EEAD1BD
:107EE00027498B88002BC6D0887909A9237801916E
:107EF00061780091310000F0EAF8BCE7002302AAA3
:107F000093833000617809AAFFF72AFFB3E71D4B7E
:107F10000993F6E7042B02D09A1F012AABD8184A1E
:107F2000043B9B00995A0029A5D0D21890783100C3
:107F30003A0000F0AEF800289DD13B88042B03D016
:107F400001213000FFF724FF012C04D1A86800288C
:107F500001D003F0EDFA280003F0DAFA8020039B49
:107F60000002434018000DB0F0BD012800D182E7A7
:107F700001213000FFF70CFFEDE7C046E867FF1F67
:107F8000D867FF1F010017000B7803704B78437010
:107F9000CB788A781B021343438070470A8803001A
:107FA00002700A88120A42700A88012A06D14A8899
:107FB00082704A88120AC2700420704702208242EE
:107FC000FBD14A8804309A704A88120ADA708A888B
:107FD0001A718A88120A5A71EFE710B5040001205D
:107FE00082420CD94B780A781B02134323808342C8
:107FF00006D1CB788A781B0213436380002010BD22
:10800000022BFBD1CB788A781B02134363804B7918
:108010000A791B021343A380F0E70B8803700B88D7
:108020001B0A43704B8883704B881B0AC3708B8874
:1080300003718B881B0A4371CB888371CB881B0A21
:10804000C3710820704703000120082A14D14A7820
:108050000878120202431A80CA7888781202024312
:108060005A804A790879120202439A80CA7988793B
:10807000120202430020DA80704710B5040001208C
:10808000022A05D100204B780A781B021343238073
:1080900010BDF8B5060010200F00150003F040FBDE
:1080A00004000120002C0ED0A0230C2229002380E4
:1080B0006780201D002D07D003F0CAF92100300091
:1080C00003F016FC0020F8BD03F0DAFAF6E7F7B586
:1080D0001E00009008AB142017001D78019103F0DA
:1080E0001FFB041E12D0A2230370019B4770438024
:1080F000099B057146710C220830002B07D019002E
:1081000003F0A6F92100009803F0F2FBF7BD0999EE
:1081100003F0B6FAF6E737B5041E0FD04388002BFC
:108120000CD00025C1881323007A172201950095F1
:10813000FFF7CDFFFF2365806372257037BD000018
:1081400010B50C4904004A88002A09D08B89002BFD
:1081500005D00020CB8A0222834201D010BD01222B
:1081600013000A20434300204032C854C8184280FC
:108170000472F3E7BA67FF1F002343800370704760
:10818000094B00211A0010B55C88002C06D01C7920
:10819000844203D10A234B43D01810BD01310A3366
:1081A0000329F1D10020F8E7BA67FF1F10B50400DA
:1081B000407A03F02DFAFF23637210BD704704303C
:1081C00010B580B203F014F9002803D0042149420D
:1081D00003F016FC10BD000070B50025104CA0681F
:1081E0002580A581A580A84202D003F0A1F9A56051
:1081F00000250C4C0C4B606D1D80230058331D7006
:10820000A84202D003F094F9656500256068002853
:1082100001D003F08DF9013508340A2DF6D170BD77
:108220008068FF1F2468FF1F7468FF1F70B5041E5D
:1082300009D1054D2880A881A880A868002802D00F
:1082400003F076F9AC6070BD8068FF1FF0B54B8815
:1082500085B00193002343600A7905000F00022ACC
:1082600000D07BE0CA88032A17D98B685E7819781A
:108270003602DC78D8790E4399781B7A24021B02E7
:108280000C43034353495BBA0B80331D93421ED109
:10829000042C04D0631F022B0ED9012015E0019A93
:1082A0004D4B1201D35A002B06D00198FFF7BEFFA9
:1082B0004A4A1369013313610421B8682E812C8066
:1082C000494203F09DFB6860002005B0F0BD434DBE
:1082D000042C06D0631F022B0FD9EB680133EB602F
:1082E000DBE7019A3C4B1201D35A002B05D00198D1
:1082F000FFF79CFF2B6901332B61374B3000029352
:10830000019B029A1B010193002301998C468B5219
:10831000130063449C8003939E81FFF750FF039BEF
:10832000041E986016D00421B868494203F068FB27
:10833000FA880100043A200003F08AF80199029AB1
:10834000FB888A5A043B9B18029A8B522B68013394
:108350002B60A2E7AB690133AB619EE71E4B029332
:10836000019B1E01029BF35A002B2DD002998C1900
:10837000A068002828D0012A26D1FA889B189BB231
:108380007352A189994217D39B1AC018B96803F098
:108390005FF8029BA289F35A934200D07DE7002246
:1083A0002B81A3882B80A3686B60029BF2520B4A3F
:1083B00053680133536070E7084A93680133936050
:1083C0000198FFF733FF68E7044A536901335361AB
:1083D000F6E7C046EA67FF1F8068FF1FF067FF1FD0
:1083E00070B5051E15D10B4C0B4B1880230058336C
:1083F0001870606D002802D003F09AF865652500BA
:1084000050356068002801D003F092F80834AC427F
:10841000F7D170BD2468FF1F7468FF1FF0B5170007
:10842000A12285B0920001934243394B06001B689C
:108430000C009B18D933FF331D78FDF741FF043042
:10844000854204DD3000FDF73BFF0430C5B2BD427C
:1084500007D33A0000213000019B03F031F805B04A
:10846000F0BD2900380003F03BF92300C6B25033B9
:108470001E700393019B29006365380003F070F9B7
:10848000CBB20293002B02D0039B01361E70002654
:108490002300503303931B78B34204D8606D002847
:1084A00031D10020DBE7029A2800002A04D0013BEA
:1084B0001000B34200D02800F700E719387003F02D
:1084C00017F8786000280ED03A78019902F0C0FFC2
:1084D000019A3B780136D3180E4A0193D369F6B25C
:1084E0000133D361D4E7039B18706065A74205D1BF
:1084F000084A1320D36A0133D362B0E7606803F0FF
:1085000017F80834F2E703F013F800236365C8E7AF
:108510003409FF1FF067FF1FF7B50D0007000421A6
:10852000686803F06DFA2B89040003702B891B0A1D
:1085300043702B8883702B881B0AC3702E890225F9
:108540000436F6B2FB2E15D81B4B9F4214D10C20DB
:1085500003F0E6F81135011E0CD0902303708E3B1A
:108560000371043B4380154B8460C680187803F088
:10857000BFF900252800FEBD5C237B43104AD318B9
:108580000093583301931B78002B0FD10300320066
:1085900038000099FFF742FF019B05001B78002B74
:1085A000E8D13800009903F0DBF9E3E7054A072535
:1085B000536A01335362DDE7FEFF0000E867FF1FE7
:1085C0002468FF1FF067FF1FF0B587B000901720E9
:1085D0000F0016000193FFF7F2FD1325041E19D0BA
:1085E0000C98031E02D00199201D9847030AE370DE
:1085F000052302AAA070043090812770009866704D
:1086000003A993800494FFF787FF051E02D0200082
:1086100002F08EFF280007B0F0BD0000F0B587B073
:108620001F000CAB1B780391059301210DAB0600D5
:108630001C78049200F0D6F81425002821D02000E0
:10864000FFF77EFD0135041E1BD01149059B0A78FA
:1086500003700132D2B2131EC68001D101231A0069
:108660000B7022713000049B03990097FFF7ACFF59
:10867000051E09D1230021000648074A093303F0EB
:10868000E7F9280007B0F0BD002363802370F8E706
:10869000EC67FF1F1781001130750000F8B5050069
:1086A0000E00064C064F2368002B02D03100280034
:1086B00098470434BC42F6D1F8BDC0469068FF1F0D
:1086C000A468FF1F0123064A5B42538000231371F5
:1086D0005362044A136053609360D3601361704720
:1086E000A468FF1F9068FF1F0200002310B5064911
:1086F0009C000859002801D1625010BD0133052BA0
:10870000F6D11320F9E7C0469068FF1F034A53884B
:10871000181A43425841404210407047A468FF1F56
:10872000F0B585B002930AAB1F780CAB1B880090A4
:1087300008000E0001920393FFF7E8FF05001120E7
:10874000002D1BD10E48FFF7E1FF04001520002C7F
:1087500014D006220B99A771E01D02F079FE019B4F
:1087600030002371029B29006371009B6680237097
:10877000039B6562E381FFF791FF280005B0F0BD20
:10878000FFFF000010B5FFF7C1FF04000220002C1E
:1087900012D060880121FFF781FF606A002801D0B4
:1087A00002F046FF28220021200002F069FF012389
:1087B00000205B426380207110BD000030B5074A85
:1087C000074C5588010013780020A54204D05B1A9D
:1087D00059424B415842104030BDC046A468FF1F6B
:1087E000FFFF0000084A10B501230C00904208D09A
:1087F000FFF78CFF031E04D0037923405A1E9341D8
:10880000DBB2180010BDC046FEFF0000024B187915
:10881000431E9841C0B27047A468FF1F70B50400A2
:108820000D001600FFF772FF002804D10D4B9C428B
:1088300000D0143070BD416A03790520002907D0AB
:1088400012221A40102A02D10520002EF2D10F2048
:10885000DB06EFD5897E0C20A94289414942494275
:108860000840E7E7FEFF0000030010B5002800D134
:1088700010BD0348034A41889142F9D09847F7E771
:10888000A468FF1FFFFF0000002330B5C45CCD5C6F
:108890006C40D4540133102BF8D130BD0F2300228B
:1088A00010B5C45C64002243CA54C25CD209013BC7
:1088B000F7D210BD0200010010B52032103102F0D5
:1088C00017FF10BDF0B58BB0039010200593170073
:1088D000049102F0ADFF0090102002F0A9FF009B70
:1088E00013240190002B05D000280CD113240098EC
:1088F00002F09EFE019B002B02D0180002F098FEB1
:1089000020000BB0F0BD102002F092FF06001020F6
:1089100002F08EFF13240500002E00D1AEE00028E7
:1089200019D01022002102F0ABFE3200290003987A
:1089300002F0DEFE041E0ED133787F2B51D83000BA
:108940000099FFF7ABFF009B1B787F2B53D8019951
:108950000098FFF7A3FF300002F06AFE002D02D05E
:10896000280002F065FE002CC1D1102002F060FF4B
:108970000600102002F05CFF0290002E7CD0002840
:1089800078D03A000F3223000125121105D00F33A1
:108990003B4015B25A4253411BB26A1E1201002BD2
:1089A00033D0049BD2B298180099029AFFF76CFF5B
:1089B000013D10220021300002F062FEADB2049FA2
:1089C0002D017D19AF4242D0002C33D0300002F08F
:1089D0002FFE029B002B00D189E7180002F028FE31
:1089E00085E729003000FFF759FF28002549009A44
:1089F000FFF74AFFA7E729000098FFF74FFF28007D
:108A00002049019AFFF740FFA5E70F210F40049985
:108A10008A18D9B28F4208D9D15C06A819540133FB
:108A2000102BF6D1029A0199C0E7791A48424141C8
:108A3000C901F2E73900300006AAFFF725FF32002E
:108A4000039806A902F054FE10370400BAE7002C80
:108A5000BCD13000029906AAFFF716FF320006A922
:108A6000039802F045FE082204003100059802F048
:108A7000EFFCABE71324A9E71324AAE7002800D0F2
:108A80006EE733E7D8BC0011F0B58BB00F001600CD
:108A90000225009000283FD0002A3DD00B1DDBB2FC
:108AA0001800029302F0C4FE1135041E34D0FDF705
:108AB00047FD05003A000099201D02F079FFEBB256
:108AC0000393E3702B0CDBB22F0A00936370FFB2A9
:108AD0002B0E2370A7700193FDF72CFD10220100CF
:108AE00006A802F065FF2100029A04AB06A8FFF772
:108AF000E9FE051E0DD1039B08223370009B04A9DB
:108B0000B370019B7770F370301D02F051FFFDF7D9
:108B10001DFD200002F08CFD28000BB0F0BDF0B56B
:108B20008FB00D00149E039004920593002A03D188
:108B3000022420000FB0F0BD002EF9D00398FFF7FB
:108B4000E5FD1424071EF4D07278337812021A431C
:108B5000B3781B041343F27812061A43036A019296
:108B6000934201D30133E3D1002D03D03B7901249B
:108B70009B07DED50822002106A802F081FD059B97
:108B800013240433DBB21800029302F051FE051ED9
:108B9000CFD0059A0499043002F00AFF0422310074
:108BA000280002F005FF3900102210310AA802F057
:108BB000FFFE2900029A06AB0AA8FFF783FE041EF7
:108BC0000FD1082206A908A802F0F2FE0822311DE2
:108BD00008A802F035FE012807D101990398FDF796
:108BE000C9FC280002F024FDA3E70124F9E70000F6
:108BF00070B51C4C05002368181E10D0002D14D130
:108C00001A78002A0CD1981C083202F021FC02F0DC
:108C100007FF0135002808D123681D70012070BDB1
:108C20000A331800082202F013FC2368002BF5D049
:108C3000122002F075FD061E0DD0C12321680370BD
:108C4000457002311022023002F002FC236831002C
:108C5000587802F04DFE206802F0EAFC0023236001
:108C6000DCE7C046CC68FF1FF8B504002020FDF704
:108C700055FB0D4EA700BB590500002B0DD0002859
:108C80000BD0D878FF2809D108492A000C55F35990
:108C900007480333611802F0DBFEF8BD290002F03B
:108CA0007FFE0028F0D1F8E7E868FF1FD068FF1FBB
:108CB000C19E001170B5064D84006359002B05D08C
:108CC000D87802F0A5FCFF226359DA7070BDC04667
:108CD000E868FF1F70B506008CB00C00150000217D
:108CE0003022684602F0CCFC31001022684602F0C7
:108CF0005FFE1D2021000322684402F059FE6846F1
:108D0000FFF7D8FD2D21040003222800694402F05A
:108D10004FFE20000CB070BDF0B50700160097B0F4
:108D200001931CAB1D7830221EAB00910AA80021D4
:108D30001C7802F0A5FC102239000AA802F038FEC7
:108D40001022002102A802F09BFC0722310002A899
:108D500002F02EFE072202AB9818631E9C41019977
:108D600002F026FE02AB9C732B005A1E934102AA0E
:108D7000D3730021102206A802F082FC06221D995E
:108D800007A802F015FE1A2002ABC01806221F9990
:108D900002F00EFE102200990EA802F009FE102229
:108DA00002AB0EA908781C78013A6040D2B2087074
:108DB00001330131002AF5D10AA8FFF77BFD10220B
:108DC00012A904000EA802F043FB102206AB0EA964
:108DD00008781D78013A6840D2B208700133013139
:108DE000002AF5D10AA8FFF765FD04431022209858
:108DF000E4B212A902F0DCFD200017B0F0BD70B59E
:108E00000E0014008CB00100102268461D0002F014
:108E1000CFFD3100082204A802F0CAFD210008227B
:108E200006A802F0C5FD6846FFF744FD04001022C5
:108E3000280008A902F0BCFD20000CB070BDF8B5F8
:108E400006000D0000243719AC4200D3F8BD02F033
:108E50003FFC030A3B70631CDBB201379D4203D920
:108E60000234F054E4B2EEE71C00EDE773B50600FF
:108E70000C000225002819D0002917D0032101A8D1
:108E8000FFF7DDFF6B469A793F231A400133134306
:108E90006A463000937101A92200FFF71BFF051EEF
:108EA00004D10322E01C01A902F0D2FA280076BD09
:108EB00003785807DA08C00FD20080009B071043E0
:108EC0009B0F1843C0B2704707230B40C908C90065
:108ED0000B4303707047000070B50400FFF7EAFE13
:108EE000134DA4006359002B21D0186A002801D02B
:108EF00002F09EFB2B59986E002801D002F098FBDF
:108F00002B59D86E002801D002F092FB2B59186F14
:108F1000002801D002F08CFB2B59586F002801D09B
:108F200002F086FB285902F083FB00232B5170BD11
:108F3000E868FF1F0E4B8000C35870B50C00002B73
:108F40000FD09D68002D0CD02B78201D0B706B78F6
:108F50004B70A97CFFF7B8FF2B7E23726B69E3602F
:108F600070BD10220021200002F08AFBF8E7C04605
:108F7000E868FF1F014B18607047C046E468FF1F98
:108F8000074A03008000825810B5002A06D0D08816
:108F9000984203D1012901D1FFF79EFF10BDC046C1
:108FA000E868FF1FF0B5264E95B087000B93BB59BC
:108FB0000500099112200A92002B31D0D888FFF7C2
:108FC000A5FB04001420002C2AD0280010A9FFF7CC
:108FD000B1FFBB591E781D6A002E23D00895FDF7FE
:108FE000EFFA07000020FDF7F1FA0790A379E61DDC
:108FF000069310AD0CA9089800F0E2FA0EA928001B
:1090000000F0D7FA0B9B0A990493069B09980293E8
:10901000079B0396019300970EAB0CAAFFF77CFE0B
:1090200015B0F0BDFDF7CCFA06903000FDF7CEFA92
:10903000E31DA779079310AB06000893DAE7C04653
:10904000E868FF1F30B50C4C85002A59030085B035
:109050000120002A0ED018006946FFF76BFF2B593C
:109060001A78D888054B002A00D1054B6A4607219B
:1090700000F0D9FB05B030BDE868FF1FB3950011C3
:10908000C195001130B5094C8500295985B01022D1
:109090006846253102F0DCF92A591121044BD088A9
:1090A0006A4600F0C0FB05B030BDC046E868FF1F4F
:1090B0005D96001130B5094C8500295985B0102204
:1090C0006846353102F0C4F92A591121044BD08881
:1090D0006A4600F0A8FB05B030BDC046E868FF1F37
:1090E0009B960011F7B54D4F86001020F4590D00E6
:1090F00002F09EFBF3592062186A132200286CD0FC
:10910000033A29009C6802F0A3F9F3591A780192F6
:10911000002A58D11E6A227D317B9446514001229B
:10912000019F114201D167461740217D9143394388
:109130002175377B4F40BC4660460027800701D42D
:109140004F081740012102208F40227D82433A437D
:109150002275377B5740BC4660460027400701D444
:1091600097080F400420227DBF0082433A432275B6
:10917000627D002794466046727B42400A4201D1DC
:1091800067460F400121627D8A433A436275777BCF
:109190005740BC4660460027800701D457080F405F
:1091A0000220627D7F00824317436775767B002231
:1091B0007E40760701D4BA080A400426617D9200F9
:1091C000B1430A4362756A78002A08D06278002A9F
:1091D00005D005220533DA7700221000FEBD0422F7
:1091E0002979114205D1A17C114202D10533033AFC
:1091F000F1E7019A21782C78002A02D10A00210097
:10920000140018220429E8D8042CE6D8052060436D
:10921000034A05331218525CDDE7C046E868FF1FB9
:10922000E8BC001110B50A001121024B00F0FBFA56
:1092300010BDC046F79600110B0030B587B001ADE8
:109240002B806B4604001100981D082202F000F9E3
:109250002A000B212000024B00F0E5FA07B030BDD8
:109260001F97001110B50A001121024B00F0DBFA24
:1092700010BDC0467397001113B50B0011006A466C
:1092800013706B4604000622581C02F0E1F86A468F
:1092900008212000014B00F0C6FA13BD939700117E
:1092A00010B50A001121024B00F0BDFA10BDC046F6
:1092B000E39700117FB505000B4BAA00D4580800B6
:1092C000002C0FD0666F237FE28821780396266FEB
:1092D0000296E66E0196A46E0094FDF709FC280044
:1092E000FFF7FAFD7FBDC046E868FF1F10B51721E4
:1092F000FFF7E0FF10BD000070B50A000D00064B3F
:109300000221040000F08FFA060029782000FFF700
:10931000D1FF300070BDC046C396001170B586B055
:1093200000236A461370836804001D78681E0A28AB
:1093300059D801A902F02CF9060633373B3F4347C1
:109340004B4F5300180000F042F9062312284BD06F
:1093500000281BD16088FFF7D9F90823002813D013
:109360004279002A47D1264B1A78072312070BD5DA
:10937000244B1A680723002A06D01668002E03D053
:10938000290001AAB04703006A4613706B461B7898
:109390006088002B2AD1FFF767FC06B070BD18006B
:1093A00000F06CF9D4E7180000F087F9D0E7180056
:1093B00000F093F9CCE7180000F0ADF9C8E7180009
:1093C00000F0C3F9C4E7180000F0F6F9C0E7180090
:1093D00000F0F6F9BCE7180000F013FAB8E718003F
:1093E00000F013FAB4E707236A46137069466088F1
:1093F000FFF782FFD1E70523012AC5D1024BB8E769
:109400007567FF1FE068FF1FE468FF1FF8B52C4F6A
:109410008600F35904000D00002B40D0DA88824208
:109420003DD15A78062A33D11A78002A2ED001204D
:1094300099681A6A097D014206D0157B054203D05E
:1094400007225A700120F8BD0220014204D0157B8A
:10945000054201D00922F4E70420014204D0127B26
:10946000024201D00B22ECE7164B1B68002BE9D01F
:109470005B68002BE6D020009847BB5900215B7841
:10948000122BDFD12000FFF715FFDBE70E4BECE7D7
:10949000112A04D1002900D032252900F2E7002D3D
:1094A00008D12000FFF732F9002803D010230279F9
:1094B0001343037121002800FDF798FAC2E7C04664
:1094C000E868FF1FE068FF1FE468FF1F70B50E4EDD
:1094D0008500AB590400002B13D01B78002B11D151
:1094E0000A4B1B68002B04D05B68002B01D02000C6
:1094F000984773595B78122B03D100212000FFF7A6
:10950000D9FE70BD024BECE7E868FF1FE468FF1F5F
:10951000E068FF1F094B8000C3581020002B0CD0BF
:109520001A6A002A09D09B68002B06D0127A1B7E8B
:10953000101C9A4200D9181CC0B27047E868FF1F7F
:1095400070B503000D0014000220002A30D000295D
:109550002ED013700B78081D53704B789370FFF763
:10956000A7FCE070012002212B7A23716B7B034062
:1095700063716A7B0A401343042263716E7B164059
:10958000334363716E7BF608F600334363712B7BC4
:109590000340A371287B014000200B43A371297B6A
:1095A0000A401343A3712A7BD208D2001343A3714C
:1095B00070BD10B50A0001000120FFF7C1FF10BD0A
:1095C00010B50A0001000220FFF7BAFF10BD70B508
:1095D00006000C000220002E30D000292ED0737817
:1095E000201D0B70B3784B70F178FFF76DFC0122F2
:1095F0003579257271794B10080013409340104063
:109600000343881010408000C9080343C9000B437E
:109610006373B1794B10080013409340104003432B
:10962000881002409200C9081343C9000B4321204F
:109630002373FCF773FE854201D2122070BD2220F5
:10964000257AFCF76BFE8542F7D823781820042B87
:10965000F4D86378012BF1D80020EFE7030010B5B0
:109660000220002909D0002B07D00322481C0A70D1
:1096700019000D3201F0ECFE002010BD03000222A3
:10968000080010B5002B06D0002904D00E32591C5A
:1096900001F0DEFE0022100010BD030010B5022014
:1096A000002909D0002B07D00422481C0A70190099
:1096B0000C3201F0CDFE002010BD10B5FFF7DEFF2B
:1096C00010BD03000220002906D0002B04D0052283
:1096D00000200A701B784B70704703000220002B9B
:1096E00008D0002906D05B7800200B70013B082BC6
:1096F00000D918307047030010B50220002909D0A6
:10970000002B07D00622481C0A7019000A3201F00B
:109710009FFE002010BD10B5FFF7B0FF10BD020086
:109720000B00022010B500290ED0002A0CD0072112
:109730001970118859701188090A99701118082236
:10974000D81C01F085FE002010BD03000A00022095
:1097500010B5002B0CD000290AD09978587809024E
:1097600001431180901CD91C082201F071FE0020D9
:1097700010BD030010B50220002909D0002B07D02E
:109780000822481C0A701900921801F061FE00209E
:1097900010BD02000B00022010B500290BD0002ADA
:1097A00009D009211970117818185970511C062216
:1097B00001F04EFE002010BD10B5FFF75FFF10BD99
:1097C00002000B00022010B5002A09D0002907D0A2
:1097D0005178197011180622581C01F039FE00202A
:1097E00010BD030010B50220002909D0002B07D0BE
:1097F0000A22481C0A701900063201F029FE0020D6
:1098000010BD10B5FFF73AFF10BD02000B0002209B
:1098100010B5002A06D0002904D018005178FFF7AF
:1098200053FB002010BDF0B585B017001E006A463E
:1098300006230500080091819380FEF7C0FC1324E5
:10984000011E02900CD03800B047041E05D128003C
:1098500001A9FEF76FFA041E02D0029801F068FE1B
:109860002800FFF701FA200005B0F0BDF0B50400B4
:109870008BB0019115000021102202A801F000FF19
:10988000334EA700B85900283CD0C388A34239D131
:109890000378002B36D14278062A18D10200010045
:1098A000553235310C3006ABFFF7A9FA002829D123
:1098B0002000FFF72FFE020006A902A801F0C8FD54
:1098C000200002A901F0CCFF01200BB0F0BD816E99
:1098D000002917D00B8A112A28D19D420ED1019858
:1098E0001231093A01F0ACFF012807D1BB59200021
:1098F0009D6EFFF70FFE29000200DEE732212000F7
:10990000FFF7D8FC2000FEF701FF061E1BD0416ABE
:10991000002918D00B8AAB4215D1082201981231C8
:1099200001F08EFF01280ED1716A0AE09D42E9D153
:1099300008220198123101F083FF0128E2D1BB59BE
:10994000996E8A7EB9E7200001F05AFFBCE7C04655
:10995000E868FF1FF0B56B4D87007E5985B03378FE
:1099600002900393002B00D087E0B368346A019320
:109970007078062817D101221B7D134202D0217B6B
:10998000114218D10222134202D0217B114251D13F
:109990000422134203D0237B134200D08BE0019BAF
:1099A0005A7DEB5991E007380428F8D801F0F0FD12
:1099B000032E42678300B36E002B03D11C2001F0FD
:1099C00037FFB066EB599C6E002C1CD01022002192
:1099D000200001F055FE0298FFF79CFD01002000D9
:1099E000FFF72DFA01F074FE2082200008211230CA
:1099F000FFF725FA0298FFF78DFDA076EB592100BD
:109A0000D888FFF70FFC0822EB591CE0B36E002B3F
:109A100005D01A00198AF0881232FFF70DFC0222D5
:109A2000019B197DEB5911423DD0207B10423AD069
:109A3000073208E0F488FCF7DBFD01002000FFF7A7
:109A400011FC0A22EB595A70029B9C002A59537848
:109A5000073B042B11D8D088FEF758FE00284ED0C3
:109A6000C3895A08D2182849029B0298CB542B5913
:109A700041180433254801F0EBFF05B0F0BDFCF7B9
:109A80009FFD03000120834201D100200393EB5985
:109A9000DE88FCF79BFD039902003000FFF7ECFB2A
:109AA000019AEB59117D042211420CD0217B114205
:109AB00009D00B22C7E7F688FCF73CFD0100300017
:109AC000FFF7EEFB6BE7019A527D01210A4204D0B9
:109AD000607B084201D00C22B5E702210A4204D083
:109AE000607B084201D00E22ADE704210A4204D077
:109AF000627B0A4201D01022A5E71222A3E7FA22D4
:109B00005200B0E7E868FF1FEC68FF1FCB9E001112
:109B100010B5064B1A780423100018401A4200D0E2
:109B20000348FFF727FA002010BDC0467567FF1FE6
:109B30000446FF1F70B50400FFF7D4FA051E43D199
:109B40002000FFF77FFA234EA400A0598268937C7F
:109B5000DB0708D50321036A1B790B40012B02D1D7
:109B6000017F0B430377431DD97F8B1E022B0DD83A
:109B7000022900D00121C088FCF790FF042133594D
:109B80001A7F59700A431A77280070BD01290CD139
:109B900002231022437000210C3001F071FD305976
:109BA00010213530FFF74BF9EEE70529ECD1022300
:109BB000D118437010220C3001F04AFC04233259B2
:109BC000117F0B431377EAE708251828DCD1053D00
:109BD000DAE7C046E868FF1FF0B58BB0059143880F
:109BE0007E4F9E00F45915000493002C15D10129D5
:109BF00002D000200BB0F0BD101D57781678FFF78B
:109C000057F9EB68320002932B7A04990193009084
:109C10003B002000FCF70CFFEBE7E388049A93423B
:109C200001D00820E6E72378012B00D1D4E0059B82
:109C3000581E092800D9CFE001F0AAFC05CE0A2958
:109C4000CC506C859AB229000498FFF773FFD1E7D6
:109C5000200029001022453001F0FAFBB9594B7859
:109C6000042B02D1013B4B70C3E70B000A002533E4
:109C700035320C310498FFF795F90498FFF702FA92
:109C80000522431E9841BB59C0005A70B2E720001C
:109C900029001022553001F0DBFB049B4F4C9D0046
:109CA000295904980A0006AB55320C31FFF77AF9AE
:109CB00029591022453106A801F0C2FD012808D11A
:109CC0000498FFF7F7F90590002804D106222B59D4
:109CD0005A7005988EE708230593FAE763780C2BF2
:109CE0007AD1E36E002B03D11C2001F0A1FDE066C8
:109CF000BB59D86E00286FD01022290001F0A8FBB4
:109D0000BB590498DC6EFFF705FC0D22A076BB5909
:109D10005A706EE7E06E00285ED063780D2B5BD141
:109D20002B8808220382A91C123001F091FBBB5939
:109D30009A68517D0222114226D0186A407B104257
:109D400022D00C32E4E763780E2B45D1236F002B31
:109D500003D1162001F06CFD2067BB59186F002855
:109D600003D01022290001F073FB0F22BB59CFE76B
:109D700063780F2B30D1206F0622691C103001F060
:109D800067FBBB599A68517D0422114203D0196ABE
:109D9000497B1142D5D100210498FFF78BFA28E7BF
:109DA000636F002B0DD0BB59586F0028F3D01022E1
:109DB000290001F04DFB0122BB5952425B6F1A6131
:109DC000E9E7142001F034FDBB5960675B6F002B9D
:109DD000E9D126E72978DFE707200BE7E868FF1FCE
:109DE00010B5064C207001F06BFD06212078FDF7C0
:109DF00091FF0348FEF778FC10BDC046FB68FF1FCB
:109E0000818F001100200BB270B50D00834216DA6D
:109E1000264B187801F0BCFD041E0DD00378922B60
:109E20000ED0A02B37D0224B1878FF283AD0210033
:109E300001F05EFD002835D180200002684070BD31
:109E400043780E2B0BD03E2BEDD18378052B12D00F
:109E5000082BE8D181798088FFF7D8FA08E0154B04
:109E600082889A42DFD183681878591CFEF7C0FEB9
:109E7000002817D1D7E7104B1B785B0712D50F4B83
:109E80001B68002B0ED09B68002B0BD0C289811D54
:109E900080889847ECE7FFF741FAA068002801D0D6
:109EA00001F046FB200001F033FBC5E7FB68FF1F14
:109EB000FD45FF1F182000007567FF1FE468FF1FA6
:109EC00010B50078FFF712FA10BD10B50078FFF753
:109ED000FDFA10BD0C234343084A10B59B185A687D
:109EE000002A03D0012901D1904710BD9B68002BA7
:109EF000FBD00029F9D19847F7E7C0461869FF1F42
:109F000001238340094A10B5946B1C439463506B42
:109F100098435063D46B20009843012901D120005D
:109F20001843D063116B0B43136310BD00800040D6
:109F3000F0B500240127154B85B0DA6B144E03925F
:109F40001A6C0192DA64019BE3403B4217D0039DF7
:109F5000E5403D400295E5B202992800FFF7BAFFBF
:109F6000316A736A002908D03900002B01D00299A8
:109F700079402800FFF7C4FF01E0002BF9D101343C
:109F80000C36172CDFD105B0F0BDC0460080004074
:109F9000FC68FF1F064B01215A68C2400A4204D0E8
:109FA0001B68C3401800084070471B6DF9E7C046A6
:109FB000008000400122064B8240002903D0D9686E
:109FC0000A43DA607047D9689143D960FAE7C0461E
:109FD0000038004030B5032444430F4BE25C1B19AA
:109FE0009C785D7801232D1B0135AB40013BA340DC
:109FF000A140DB430C00122807D8084992005218F0
:10A00000116819402143116030BD054A11680B40A9
:10A0100023431360F8E7C0462FBD001108F000404D
:10A0200014F00040C21F70B5D4B20623092C0BD81F
:10A030000125084C9540002908D00021FFF7CAFFF0
:10A0400023682B4323600023180070BD2368AB43B3
:10A05000F8E7C04600380040214BF0B51B185B788C
:10A06000022B21D1032444431E4A1F4EA35C121924
:10A070009478012215008540B76B013CE4B23D4362
:10A08000A240B563194C122815D89B0000290CD1A9
:10A0900017495B1899680A439A600123205C154AA6
:10A0A000834011680B431360F0BD11495B18996838
:10A0B00091439960F1E70E4B00290DD159690A438C
:10A0C0005A61225C1328E8D00123203A93400A49C0
:10A0D000086803430B60E7E7596991435961F0E76A
:10A0E000FC68FF1F2FBD00110080004074BD0011EF
:10A0F00000F00040A0F00040A4F00040F8B50024BB
:10A100001B4E1C4D1C4B1B5D012B1FD1194A926924
:10A11000E2401A420BD00122B25693402200143A78
:10A12000D2B2022A09D815494A6913434B61013456
:10A1300002360C35172CE5D1F8BD0022B2560F4976
:10A140009200521891680B439360F0E7022BEED116
:10A15000E7B23800FFF71EFF01235840C1B23800B4
:10A16000FFF77AFF3800FFF715FF6877DFE7C04693
:10A1700001BD0011FC68FF1FFD68FF1F00F00040DB
:10A18000012202388240054B002903D059690A4355
:10A190005A617047596991435961FAE700380040A4
:10A1A000F8B50E0001210F008740114A0400D36862
:10A1B000FD43BB43D360831E8B4201D8FFF7E0FF12
:10A1C00000212000FFF72EFF0A4A0B4B5168012E99
:10A1D00005D139431B1951605E700020F8BD29403C
:10A1E000516002221C1962709A6915409D61F4E762
:10A1F0000038004000800040FC68FF1F012210B5BD
:10A200008240074B002906D019680A431A600121D1
:10A21000FFF7C6FF10BD196891431960F7E7C04604
:10A22000008000400C2370B5002543430A4A2900F2
:10A230009B181D70094B04001B185D70FFF7B0FFE1
:10A240000123A340064928000A681A430A60054909
:10A250000A689A430A6070BD1869FF1FFC68FF1FF7
:10A26000348000403080004070B504000E00FF28AC
:10A2700013D003250540FFF7D5FF084AA3089B002C
:10A280009B183F22ED00AA40AE4019682000914380
:10A29000314319600121FFF78DFE70BD1838004071
:10A2A000F8B50C244443134B0500E4186368002BF5
:10A2B00003D1A3681220002B1AD0022201270E4BD3
:10A2C00000215B195A7028002770FFF769FF636847
:10A2D0001E1E08D0A3683E00002B04D02800FFF704
:10A2E00059FE4640F6B228003100FFF709FE002073
:10A2F000F8BDC0461869FF1FFC68FF1FF7B5C420F2
:10A30000FF222B4B80001958002491433F3A0A4307
:10A310001A508022274F5202274E1A60274B1D5D8C
:10A32000002D21D0A31E012B03D80121E0B2FFF79D
:10A3300027FF012D18D11F4B9B69E3402B4213D0FF
:10A34000E3B218000193FFF725FE01000198FFF723
:10A3500055FFE3B2143B022B1DD801217156184A58
:10A360008D405369AB4353613B7F002B0DD0E5B269
:10A370002800FFF795FF2800FFF70CFE7B7F010008
:10A38000834202D02800FFF7A5FD01340C370236C6
:10A39000172CC3D1F7BD012100237156F3568D4010
:10A3A000074A9B009B189A68AA439A60DCE7C0465C
:10A3B00000E100E0FC68FF1F01BD0011FD68FF1F08
:10A3C00000F0004010B501210400FFF7E9FE012371
:10A3D000044A002011194B70A34091690B4393610B
:10A3E00010BDC046FC68FF1F70B50E0015000400CC
:10A3F000FFF718FF0C236343094A20009B189D6058
:10A400005E60FFF74DFFF021064B074A8900051EED
:10A410005A5002D02000FFF705FF280070BDC0464B
:10A420001869FF1F0000FF1F319F001170B5134D09
:10A4300007202C78002C1FD19822210052002800E0
:10A4400000F0EEFF0123C420FF222B700C4B800094
:10A450001C635C630B4B1C605C600B4B1958914395
:10A460003F3A0A431A50802252021A600D20074ACE
:10A47000074901F0B5FA200070BDC046FC68FF1F17
:10A4800000800040A0F0004000E100E0FDA20011CB
:10A49000FDA00011030010B50620072B09D8054ABE
:10A4A000137001F0FDF8D7210020034B034A890007
:10A4B0005A5010BD2C46FF1F0000FF1F151BFF1F29
:10A4C00070B51D0002240C2910D8094ACA40D207D1
:10A4D0000CD5FBF72FFF041E08D1059A049928001C
:10A4E000FBF744FFFCF7B2FDFFF712FB200070BD45
:10A4F0001210000030B50D7802232C009C43184246
:10A5000001D02B431C0008252300AB43284201D077
:10A510002B00234320241D00A543204201D01C43CF
:10A5200025002A230D70184204D011781E3B0B43DE
:10A53000137030BD0028FCD10C2113788B43F7E752
:10A54000F8B51D0006AB1B88140007AA0E000B20EF
:10A550001778002B27D10A78022A49D14A68507807
:10A5600011780002244A08438018042840D801F0DA
:10A570000FF803121D1B2300F06801F061FA021CA2
:10A58000C0B2B84200D93A1CD2B22000F1682A8089
:10A5900000F05EFF06E00222F3681B882A80237029
:10A5A0001B0A63700020F8BD0622EEE701232B8012
:10A5B000F3681B782370F5E7F368002B16D00822A8
:10A5C0002A801A8822701A88120A62705A88A27029
:10A5D0005A88120AE2709A8822719A88120A627165
:10A5E000DA88A271DB881B0AE371DBE72B80D9E7ED
:10A5F00001202B80D7E7C04600D6FFFFF7B5160035
:10A600000A781D0008AB1F880C000123022A18D10C
:10A610004A685078117800022B4A084380180328B2
:10A620000FD800F0B5FF02254439E06801F008FAC0
:10A63000C0B20723B84204D37B190193152B02DD66
:10A640000D231800FEBDE0682A003100C01900F09B
:10A65000FFFE6B4600209B88E268D0541B4B1B68B2
:10A66000834203D01B68834200D098470023E8E769
:10A670000B23002FE5D1022DE2D1737832781B0233
:10A680001343E2681380114B1B68002BEED01B684C
:10A69000002BEBD00120E8E70B23002FD1D1062DB2
:10A6A000CED12A003100E06800F0D2FEDEE70B23B5
:10A6B000002FC6D1012DC3D132787533012AC0D8FD
:10A6C000E3681A70D2E7C04600D6FFFF086BFF1F91
:10A6D00070B50C001500072837D800F059FF041496
:10A6E00036361B36242E182015290BD8184E162264
:10A6F0000021300000F0C4FF22002900300000F0EB
:10A70000A7FE002070BD18200229FBD11288114B32
:10A710001A80F6E718200829F4D10A000E4829000B
:10A7200000F04EFFEDE718200129EBD10B4B10781C
:10A730000B49DA69FFF7DEFEE3E718200129E1D1D2
:10A74000064B10780749DA6BF4E70220DAE7C046D7
:10A75000F06AFF1FAA46FF1FA046FF1F3046FF1FDB
:10A760005846FF1F7846FF1F030010B50020DB0787
:10A7700004D50721024A034800F08CF810BDC046FA
:10A780008CBD00113046FF1F054A030010680028E9
:10A7900003D082889A4201D1806870470068F6E74A
:10A7A0000C6DFF1F0A88030008009A4204D08A88B3
:10A7B00004309A4200D0002070470000F8B5F8221B
:10A7C00000230D4F0D4E79680500424333709942C6
:10A7D00000D07B600A4C0021200000F051FF0023D4
:10A7E0001A007C60AB4202D100203370F8BD013307
:10A7F0002280DBB2F834F5E70C6EFF1F086EFF1FF6
:10A80000106DFF1F73B56B4601900600684615007A
:10A810001980FCF74DFF041E11D1002D0FD0768951
:10A82000002E11D00C2001F003F800280ED0084AA9
:10A830000460136886808560002B02D110602000C0
:10A8400076BD1A001B68F7E70224F8E71324F6E741
:10A850000C6DFF1F012100220A4B10B549420A4C22
:10A86000198099809A719A70084B20700120198084
:10A870005A60FFF7A3FF2078FCF778FF0448FDF744
:10A8800033FF10BD106BFF1F146EFF1F0C6EFF1FF8
:10A8900041A90011022310B5002802D0FFF7B2FF32
:10A8A0000300180010BD0000030010B50020DB07F6
:10A8B00004D50421024A0348FFF7A4FF10BDC04697
:10A8C000A0BD0011B046FF1FF0B50E2687B0039360
:10A8D0000CAB1F8802ABF61805000800310002928D
:10A8E000FDF768F804000120002C0FD03088FFF736
:10A8F0004BFF03000E20002B08D05E68002E05D011
:10A9000021002800039B029A0097B04707B0F0BDD2
:10A910000A4B10B5984207D10122002352420A8007
:10A920008B708A808B7110BDFFF73CFF0028FAD036
:10A9300001235B42038000238370F4E7FFFF0000E4
:10A94000F8B5050001290AD1134E00243388F827F1
:10A95000AB4219D028001149FFF7DAFF06E00229BF
:10A9600004D10139FDF73EFF0028EDD0F8BD3B00D2
:10A9700063437268D018D35A002B09D03A000021E3
:10A9800000F07EFE0134E4B2054B1B78A342EED802
:10A9900001235B423380DDE70C6EFF1F106BFF1F4E
:10A9A000086EFF1F10B5FFF7FDFE03000020834275
:10A9B00000D0987810BD0000F0B589B01C000EAB37
:10A9C00080CB03901E8810AB1B78049202930B7A05
:10A9D0000D00DB0616D42B780593022B24D00498A7
:10A9E000FFF7D2FE002812D003689C46002B0ED041
:10A9F000029B2200019329003B00644603980096C5
:10AA0000A04705E00498FFF7BFFE002802D10E2002
:10AA100009B0F0BD8368002BF9D00A222900039801
:10AA200098470028D7D0F3E76B6858781A786B4BB3
:10AA3000000210439842D2D8043B984210D2684B8F
:10AA4000984242D015D8674BC0180128C7D80B20B0
:10AA5000002EDDD1EB681A7859683A80200028E092
:10AA6000614BC018032800D979E000F091FD846A99
:10AA7000789E5E4B9842B2D10B20002EC8D10123A4
:10AA80003B80EB6831001B7823706889013080B20D
:10AA9000FCF790FF3A88031E0ED0017802328A1824
:10AAA0003A80428962704289120AA270596802781B
:10AAB000E01C00F0CDFC06E004323A8031000422B4
:10AAC000601C00F0DDFD0020A2E70B20002E9FD1CE
:10AAD000EB6807A91E8804233B80330A30002670E8
:10AAE0006370FCF767FF051E28D004AB9A890E231C
:10AAF00004A95B183E49C668FCF7D0FF00280BD1BB
:10AB00002B783C486A680599FBF786FB002803D13F
:10AB1000012304AA5B42D3813278022A06D17168EC
:10AB2000201D00F095FC3B8802333B800E2304AAD5
:10AB30009B181B88A3701B0AE370C4E704ABDE817B
:10AB4000F4E70B20002E00D062E7E9680398FFF7D6
:10AB500029FF02233B802070000A6070B3E70B20BE
:10AB6000002E00D054E70222EB681B883A80237045
:10AB70001B0A6370A7E7E86800F062FFC2B2030037
:10AB80000720B24200D243E70DD00299DBB2711820
:10AB9000994202DB921BD3B20293029BE9681A002E
:10ABA0003B8089195AE70023F6E70B20002E00D0DE
:10ABB0002EE70722EB683A801A7822705A78627082
:10ABC0005A88A2705A88120AE2701A792271DA88B9
:10ABD0006271DB881B0AA37175E7C0460429000077
:10ABE0000228000000D8FFFFFFD6FFFF0328000067
:10ABF000FFFF0000D0BC0011F0B58DB06B46002007
:10AC0000089120229B5E83423DDAA64B187800F023
:10AC1000BFFE071E32D00378B02B2CD1007902384A
:10AC200016281FD800F024FC17001E001E001E006E
:10AC300031001E0096001E001D011E0052011E0064
:10AC400073011E00CD011E0050021E001E001E00DA
:10AC50008E021E00E302944B94491B8878880B8077
:10AC6000FBF71AF83800FCF79BFF914B1B68002B91
:10AC700001D038009847380000F04AFC8020089B3B
:10AC80000002434018000DB0F0BDF62200218748B5
:10AC900000F0F6FC0BAA3B7B7989388900923A00D8
:10ACA0000D32FCF79FFD0400804B1B78002C3FD138
:10ACB00046E0804B788805937F4B4100CB5A0BAE22
:10ACC000073BDBB232880293002301937B4B2100C8
:10ACD00006930093059BFFF76FFE744D002810D17B
:10ACE000069B3A8A1B889A420BD13800059912308C
:10ACF00000F0A6FD002804D02B7862899B00EB1899
:10AD00005A80162306A81B18328820007989FCF780
:10AD1000C5FE2B7804009A00AA1851880029C3D0D8
:10AD20000133DBB22B70002807D006A9C98A9180B5
:10AD3000634A12889A42BCD802E0012149429180BC
:10AD4000002B04D059497888FAF7DAFF8AE73E8960
:10AD50000A2479E000253E89574B06937B88069AA2
:10AD60005B009B5A033B9D4202DB002DF0D05BE071
:10AD7000162206A812183B7B798900923A0030000F
:10AD80000D32FCF72FFD0590002858D04689017A36
:10AD90007888FCF7F1FC041E44D1464B7888079371
:10ADA000069B4100C95A454B0439C9B206AAD28A4A
:10ADB00006930291019400930599079BFFF7FCFD10
:10ADC000041E2FD1069B39491A88931C002D26D1C9
:10ADD0004B807988384B4900CB5A5119033B8B4241
:10ADE00020DD059B31485B8941190B71A91C013598
:10ADF000C9B2EDB2059145191B0A2B71059B2D496E
:10AE00000433181800F024FB2C4B059A1B88D31828
:10AE1000DDB22C4B9E4205D00136B6B29CE7498884
:10AE20009942D6D0002D0CD0204C2800618800F02B
:10AE3000DFFB207021007888FAF772FF12E7059C8B
:10AE4000F0E7002C00D183E77B78142B00D109E7D1
:10AE500016493B794E800B700C717888FAF712FF17
:10AE600000E7162406ABE41821003889FCF7A2FDA0
:10AE7000011E00D1B7E1788822880F4C45002C5B79
:10AE80000A4D013CE4B2029400240F4B019400955A
:10AE9000FFF792FD041E00D014E129007888FAF72C
:10AEA0004FFFDFE6146EFF1F9C45FF1F186BFF1F4F
:10AEB0000C6BFF1F126CFF1F4867FF1F086DFF1F01
:10AEC0009A45FF1FFFFF00001A6BFF1F162406ABF9
:10AED000E41821003889FCF76DFD011E00D182E1E4
:10AEE00078882288AE4C45002C5BAE4D013CE4B224
:10AEF00002947C89AC4B01940095FFF75DFD041E24
:10AF000000D0DFE029007888FAF724FFAAE60025C0
:10AF1000A44B1D803B00FE331B78A24A7888079221
:10AF2000AB4208D99E4B12880693069943005B5AA0
:10AF3000013B9A4203DB0799FAF716FF92E61624C3
:10AF40006B00FB18059306ABE418059B21001889DC
:10AF5000FCF730FD011E03D1059B01241E8973E718
:10AF60007888924B2288069C099343001B5B904E85
:10AF7000013BDBB20293002300960193099BFFF78C
:10AF80001BFD041E02D0059B1E895DE77B88069A87
:10AF90005B009B5A079A108832881218934202DC91
:10AFA0001B1A013B33807F4C02303288099900190B
:10AFB00000F04EFA2388328801359B182380EDB2C9
:10AFC000A8E70BAA3B7B7989388900923A000D32B9
:10AFD000FCF708FC00250590059B002B04D10A24F2
:10AFE000002D00D16EE060E0059B7888197AFCF7AF
:10AFF000C3FB0100041E63D1694C6C4B7888069436
:10B000000993069B4400E45A694B063CE4B20BAE3C
:10B01000328807930294019100930599099BFFF7E9
:10B02000CBFC041E4CD1079B5E491B881A1D002DCA
:10B0300030D14A80059B5B4C5A8963191A716B1C8D
:10B040009BB2E318120A1A71162306A832881B183D
:10B0500079890598FCF722FDFF21AA1C2E1D0335D6
:10B060000B00059092B2B6B2ADB2002803D006AB89
:10B07000DB8AD9B21B0AA218651911712B714C4DCC
:10B08000301D2A884949201800F0E2F92B88F6186B
:10B09000B5B2A1E74988914207D17A880699520052
:10B0A000525AEB18053A9A42C4DC3E4C280061889B
:10B0B00000F016FB207021007888FAF75FFED1E5DA
:10B0C000002DF2D13E89BFE6162606ABF6183100F8
:10B0D0003889FCF76FFC3D000400FF3500282DD0B7
:10B0E000037A9B060CD400227B89398978880092E8
:10B0F0003A000C32FFF7E8FB041E10D03E8915E041
:10B100003088FFF741FB00281AD08368002B17D046
:10B110002100122278889847041EE4D0EEE7AB782D
:10B12000002B02D17888FAF739FE0026AB78002B85
:10B1300000D097E5002C00D194E585E60124DDE7F9
:10B140000E24DBE7162506ABED1829003889FCF73D
:10B1500031FC041E47D0037A9B0611D4154A7B8824
:10B160001188994203D01448814207D11380134BB0
:10B17000F8261D780023D9B2A94221D30924A1E7DA
:10B180002888FFF701FB00282FD08368002B2CD0E4
:10B190002100122278889847041EDFD092E7C0462B
:10B1A0004867FF1F186BFF1F1A6BFF1F126CFF1FF2
:10B1B000086DFF1F0C6EFF1FFFFF0000086EFF1FD2
:10B1C00031005943546801336018615A0029D2D1C3
:10B1D0003C0008342100F82200F03AF92100788878
:10B1E000FAF7E4FD3EE501246CE70E246AE71D4B07
:10B1F0001A887B889A4231D07888FAF7E1FD31E5E8
:10B20000F823059851684343CD18C95A00291FD027
:10B210003B7A012B0BD16C88AB887888AA1D0094EF
:10B22000FFF752FB041E02D000233B722E88F82247
:10B230000021280000F024FA00232B80059B013315
:10B24000DBB20593084B05991B78064A8B42D7D889
:10B2500001235B421380002CCED0F5E5002634009C
:10B260000596EFE70C6EFF1F086EFF1F70B5040018
:10B270000E001500FFF796FA031E08D131000548AD
:10B28000FFF790FA03001120002B02D01C80002051
:10B290009D7070BDFFFF0000F8B50B4F06003B78B6
:10B2A0000D001400FF2B0ED00A2000F039FA011E09
:10B2B00009D0B1230380002346800371C580048137
:10B2C000387800F015FBF8BDF146FF1FF7B50F0009
:10B2D00008A90600088809A90B240988002821D19B
:10B2E0000234022B1ED1557813782D021D432B00FA
:10B2F0008B4301937334002B14D1FB683000190089
:10B300000093FFF74FFB019C85420BD02A003000D1
:10B310000099FFF7ABFF041E04D12A0030007989A1
:10B32000FFF7BAFF2000FEBDF0B50E7885B00390A0
:10B330000AA805880120022E0DD14C682778647870
:10B3400024023C43054FBC4205D10398DBB2019671
:10B350000095FFF7BBFF05B0F0BDC0460229000015
:10B3600010B504000C4800F07BF90C48A16B00F00C
:10B3700077F90B48E16B00F073F90A48216C00F093
:10B380006FF9094B0948196800F06AF9084B1B6806
:10B39000002B00D09847FEE7A2BB0011B8BB0011FC
:10B3A000C7BB0011D6BB001104ED00E0E5BB0011E6
:10B3B000186EFF1F002307B501A80193FFF7D0FF08
:10B3C000044A0548002110B5121A00F059F9F8F79F
:10B3D000F7FAFEE71C6EFF1FF446FF1F0000000097
:10B3E00001B40248844601BC604700BF613BFF1FB7
:10B3F00001B40248844601BC604700BFE928000050
:10B4000001B40248844601BC604700BF2526000005
:10B4100001B40248844601BC604700BF5D32FF1F93
:10B4200001B40248844601BC604700BFB70E00006B
:10B4300001B40248844601BC604700BF851F00007C
:10B4400001B40248844601BC604700BF2D38FF1F8D
:10B4500001B40248844601BC604700BFE94C0100CA
:10B4600001B40248844601BC604700BF056A000081
:10B4700001B40248844601BC604700BFD93DFF1FAC
:10B4800001B40248844601BC604700BF9DA900008A
:10B4900001B40248844601BC604700BFDD6601007C
:10B4A00001B40248844601BC604700BFE139FF1F78
:10B4B00001B40248844601BC604700BFB54C01009E
:10B4C00001B40248844601BC604700BF5118FF1F09
:10B4D00001B40248844601BC604700BF291C00003B
:10B4E00001B40248844601BC604700BF6D30FF1FB5
:10B4F00001B40248844601BC604700BF017F0000E0
:10B5000001B40248844601BC604700BF4D1F0000E3
:10B5100001B40248844601BC604700BF434D0100AE
:10B5200001B40248844601BC604700BFC51D00004D
:10B5300001B40248844601BC604700BFD9490100FC
:10B5400001B40248844601BC604700BF0D3CFF1FA8
:10B5500001B40248844601BC604700BFEDA500006D
:10B5600001B40248844601BC604700BFF30E0000EE
:10B5700001B40248844601BC604700BF5D38FF1F2C
:10B5800001B40248844601BC604700BFC95C0100A9
:10B5900001B40248844601BC604700BFC53DFF1F9F
:10B5A00001B40248844601BC604700BF0D5201004F
:10B5B00001B40248844601BC604700BF3D1800004A
:10B5C00001B40248844601BC604700BF810E000000
:10B5D00001B40248844601BC604700BFED4A010047
:10B5E00001B40248844601BC604700BF6DBC000046
:10B5F00001B40248844601BC604700BF350E00001C
:10B6000001B40248844601BC604700BF456B01009D
:10B6100001B40248844601BC604700BF11470100E5
:10B6200001B40248844601BC604700BF5952010082
:10B6300001B40248844601BC604700BF014C0100D0
:10B6400001B40248844601BC604700BFC94A0100FA
:10B6500001B40248844601BC604700BFB3520100F8
:10B6600001B40248844601BC604700BFE53A0100CE
:10B6700001B40248844601BC604700BF2D39FF1F5A
:10B6800001B40248844601BC604700BF154D01006B
:10B6900001B40248844601BC604700BF3555000034
:10B6A00001B40248844601BC604700BF151BFF1F60
:10B6B00001B40248844601BC604700BFA13BFF1FA4
:10B6C00001B40248844601BC604700BF691F000006
:10B6D00001B40248844601BC604700BF2951010003
:10B6E00001B40248844601BC604700BF090E000057
:10B6F00001B40248844601BC604700BFE548000031
:10B7000001B40248844601BC604700BF4532FF1FB8
:10B7100001B40248844601BC604700BFF94C0100F7
:10B7200001B40248844601BC604700BF1D4D0100C2
:10B7300001B40248844601BC604700BF51250000A7
:10B7400001B40248844601BC604700BF055E0000AA
:10B7500001B40248844601BC604700BFC521000017
:10B7600001B40248844601BC604700BF090E0000D6
:10B7700001B40248844601BC604700BFADAE000082
:10B7800001B40248844601BC604700BFB14E0000CE
:10B7900001B40248844601BC604700BF9D32FF1FD0
:10B7A00001B40248844601BC604700BF2124000068
:10B7B00001B40248844601BC604700BFB53CFF1F8E
:10B7C00001B40248844601BC604700BF0189000003
:10B7D00001B40248844601BC604700BFB930FF1F76
:10B7E00001B40248844601BC604700BF79180000DC
:10B7F00001B40248844601BC604700BFC53F000059
:10B8000001B40248844601BC604700BF091B000028
:10B8100001B40248844601BC604700BF0124000017
:10B8200001B40248844601BC604700BF156B0100AB
:10B8300001B40248844601BC604700BF3D4B010093
:10B8400001B40248844601BC604700BFCD4C0100F2
:10B8500001B40248844601BC604700BF6571010025
:10B8600001B40248844601BC604700BF311B0000A0
:10B8700001B40248844601BC604700BF8534FF1F05
:10B8800001B40248844601BC604700BFB13DFF1FC0
:10B8900001B40248844601BC604700BFE93AFF1F7B
:10B8A00001B40248844601BC604700BFA54F0100B7
:10B8B00001B40248844601BC604700BF1D4B010033
:10B8C00001B40248844601BC604700BFC92600009D
:10B8D00001B40248844601BC604700BF5522000005
:10B8E00001B40248844601BC604700BF893CFF1F89
:10B8F00001B40248844601BC604700BF594F0100B3
:10B9000001B40248844601BC604700BFE117000053
:10B9100001B40248844601BC604700BF3938FF1FAC
:10B9200001B40248844601BC604700BF8D1200008C
:10B9300001B40248844601BC604700BFC9A90000A9
:10B9400001B40248844601BC604700BF8B5201002D
:10B9500001B40248844601BC604700BF8552010023
:10B9600001B40248844601BC604700BF7D18FF1F38
:10B9700001B40248844601BC604700BFC534FF1FC4
:10B9800001B40248844601BC604700BF4550000036
:10B9900001B40248844601BC604700BFF54E010077
:10B9A00001B40248844601BC604700BF5147010012
:10B9B00001B40248844601BC604700BF4551010004
:10B9C00001B40248844601BC604700BF213BFF1F11
:10B9D00001B40248844601BC604700BFC56D010048
:10B9E00001B40248844601BC604700BFE532FF1F36
:10B9F00001B40248844601BC604700BFF535FF1F13
:10BA000001B40248844601BC604700BF55490100AB
:10BA100001B40248844601BC604700BFD53AFF1F0D
:10BA200001B40248844601BC604700BFD91B000036
:10BA300001B40248844601BC604700BF5D170000A6
:10BA400001B40248844601BC604700BFDD520100DA
:10BA500001B40248844601BC604700BFA94601000A
:10BA600001B40248844601BC604700BF75A90000CC
:10BA7000000301030200030304020502060207009B
:10BA8000080309030A030B030C000D000E030F0348
:10BA9000100311001303140315031603A13D001135
:10BAA000D53D00110000000002000000B2BA0011F4
:10BAB000192A0F1809000000F1590000FD240000A8
:10BAC000F17D0011059E001159720011F57B0011E6
:10BAD00001540011F9AB001179500011913F001190
:10BAE000C140001100000000161600000200000016
:10BAF000F8BA0011F4FFF3FFD2FC0000014200117C
:10BB00000000000000000000547579610042312EF1
:10BB1000330030303031006769746875622E636FAE
:10BB20006D2F707676780054484232000200000093
:10BB300040BB0011292A282A272A262A252A242A16
:10BB40000A180000E20400007102000078EC000016
:10BB5000744000001027000060F000000664000040
:10BB6000204E000000000000050000001F501D00D6
:10BB7000023CB40000011300130000008102000029
:10BB80003031323334353637383941424344454613
:10BB9000005048592B36325858504C555330353098
:10BBA00034005B48617264206661756C7420686162
:10BBB0006E646C65725D0A004C522020203D20307E
:10BBC00078253038780A0050432020203D203078F6
:10BBD000253038780A0050535220203D20307825F7
:10BBE0003038780A0049435352203D2030782530C0
:10BBF00038780A000558001159580011000000005B
:10BC0000020000000CBC00116F2A6E2A1A180000F6
:10BC100001A00000000000006410B71DC8206E3BAA
:10BC2000AC30D9269041DC76F4516B6B5861B24D43
:10BC30003C7105502083B8ED44930FF0E8A3D6D6AD
:10BC40008CB361CBB0C2649BD4D2D38678E20AA015
:10BC50001CF2BDBDFB349B5F800000800010000023
:10BC6000000000005B5E0011E57400117F5E0011B2
:10BC7000ED780011035F0011C3780011795F0011A6
:10BC800099780011CB5F0011617A001133600011C7
:10BC9000617A0011656000111B7A0011795F001153
:10BCA00051780011F15F0011F979001100000000D6
:10BCB00000000000D7600011F9790011396100110E
:10BCC000FD740011052A042A012A002A02290328EA
:10BCD00001280028011800180000000000000000E2
:10BCE00000000000000000870101020102010102C2
:10BCF0000102030304010301010101010303020125
:10BD000003000D000E0010001100130014010701C4
:10BD100008010A010B011C011D02040205020702B1
:10BD2000080219021A021C021D0301030203170074
:10BD30000201000504000807000B0A001716001D89
:10BD40001C010201010504010E0D01111001141363
:10BD5000011716011A19020201020B0A020E0D0246
:10BD60001110021413021716030504030807030B2E
:10BD70000A030E0D0001020307090A0B0E0F101132
:10BD800012141718191A1B1F2021220041A5001197
:10BD9000FDA500110000000002000000D6BC00114B
:10BDA0000000000029B300110000000002000000A4
:04BDB000D4BC0011EE
:020000041FFFDC
:1000000000000000FD3E0011B8BA0011B4BA0011A2
:100010000064FF1F0000000000000000000000005E
:1000200000000000000000000000000000000000D0
:1000300000000000000000000000000000000000C0
:1000400000000000000000000000000000000000B0
:1000500000000000000000000000000000000000A0
:100060000000000000000000000000000000000090
:100070000000000000000000000000000000000080
:100080000000000000000000000000000000000070
:100090000000000000000000000000000000000060
:1000A0000000000000000000000000000000000050
:1000B0000000000000000000000000000000000040
:1000C0000000000000000000000000000000000030
:1000D0000000000000000000000000000000000020
:1000E0000000000000000000000000000000000010
:1000F0000000000000000000000000000000000000
:1001000000000000000000000000000000000000EF
:1001100000000000000000000000000000000000DF
:1001200000000000000000000000000000000000CF
:1001300000000000000000000000000000000000BF
:1001400000000000000000000000000000000000AF
:10015000000000000000000000000000000000009F
:10016000000000000000000000000000000000008F
:10017000000000000000000000000000000000007F
:10018000000000000000000000000000000000006F
:10019000E934FF1F3133FF1FC1660100000000007A
:1001A000000000000000000000000000000000004F
:1001B000000000000000000000000000000000003F
:1001C000000000000000000000000000000000002F
:1001D000000000000000000000000000000000001F
:1001E000000000000000000000000000000000000F
:1001F00000000000000000000000000000000000FF
:1002000000000000000000000000000000000000EE
:1002100000000000000000000000000000000000DE
:1002200000000000000000000000000000000000CE
:1002300000000000000000000000000000000000BE
:1002400000000000000000000000000000000000AE
:10025000000000000000000000000000000000009E
:10026000000000000000000000000000000000008E
:10027000000000000000000000000000000000007E
:10028000000000000000000000000000000000006E
:10029000000000000000000000000000000000005E
:1002A000000000000000000000000000000000004E
:1002B000000000000000000000000000000000003E
:1002C000000000000000000000000000000000002E
:1002D000000000000000000000000000000000001E
:1002E000000000000000000000000000000000000E
:1002F00000000000000000000000000000000000FE
:1003000000000000000000000000000000000000ED
:1003100000000000000000000000000000000000DD
:1003200000000000000000000000000000000000CD
:1003300000000000000000000000000000000000BD
:1003400000000000000000000000000000000000AD
:10035000000000000000000000000000000000009D
:10036000000000000000000000000000000000008D
:10037000B5B3001100000000000000000000000004
:10038000000000000000000000000000000000006D
:10039000000000000000000000000000000000005D
:1003A000000000000000000000000000951AFF1F80
:1003B000000000000000000000000000000000003D
:1003C000000000000000000000000000000000002D
:1003D000000000000000000000000000000000001D
:1003E000000000000000000000000000000000000D
:1003F00000000000000000000000000000000000FD
:081838002072FF1F4118FF1F81
:10184000024981F3088802F033FD00002072FF1F77
:1018500010B502F0E5FA072804D0122808D00228B3
:1018600008D010BD044A0420136B01331363F8E75A
:101870000220F6E71420F4E7F067FF1FF8B5070031
:101880000C0026002500503630785135002804D150
:101890000300287058342370F8BD2978CA00481E08
:1018A0008141A3183800A25C5B68C9B2FFF7D0FF82
:1018B00000280DD12B78DA00A218013350602B706C
:1018C0003378044A013B3370136A01331362D8E75B
:1018D0000123DFE7F067FF1F5C234343074910B58F
:1018E000C9180B0058331B78012B05D1FFF7C6FF31
:1018F000034A936A0133936210BDC0462468FF1FF8
:10190000F067FF1F10B502F07BFA064A01211300B1
:1019100010CB4942D967044B136002F099FB2000B9
:1019200010BDC04600E100E01000100010B504003A
:1019300002F066FA024B1C6002F08AFB10BDC04642
:1019400000E100E010B5040002F05AFA4021094A13
:10195000200013688B43136002F0DAFC01F0A6FD4F
:101960000022054B01201A60044B04321A6002F079
:1019700007FCFEE71CF00040C4F00040C0F000404F
:10198000431E5A425341A022F0B5D2015B4213409C
:10199000154D164A40019B182A18127E8BB00191F2
:1019A000002A1BD01A000832D46F0022E6B206AF1C
:1019B000E4B294420EDC2818C369002B08D00199C8
:1019C00002AA117106AA049202AA167303A89847E4
:1019D0000BB0F0BD1978B9540132EAE71A7D1A78D4
:1019E00006AB01261A70E6E7B06AFF1F0040004010
:1019F000F0B5254B04004001C25C85B0002A2BD015
:101A00001A18117E002927D0917E002924D011793F
:101A1000022921D11689D788D168F51BADB22A1CBD
:101A2000102D00D9102292B2BE4217D118180123EE
:101A300003710023C269C38003819A4206D06846BD
:101A4000032103730171029301A890470820002C21
:101A500000D0192001F022FC05B0F0BD013C654228
:101A60006C41A0256442ED012C40084D1B186419FF
:101A7000074D0633013A92B2AA42EDD01888461CAF
:101A80001E80085C2070F5E7B06AFF1F0040004030
:101A9000FFFF00000F220E4B10B59868104002386F
:101AA0000A280BD802F08EF90D0A0B0A0A110A0A4D
:101AB0000A0A060002210020FFF762FF10BD012183
:101AC000F9E70020FFF794FFF8E7DB6FF6E7C04681
:101AD000004000400F220E4B10B5986810400238AD
:101AE0000A280BD802F06EF90E0A0B0A0A120A0A2B
:101AF0000A0A060002210120FFF742FF10BD012162
:101B00000800F9E70120FFF773FFF7E7DB6FF5E760
:101B10000090004013B5334C2378072B3DD8324B4F
:101B20001A78324B002A39D18022196852020A43AE
:101B30001A60252001F0F4FF20232D4A11680B4381
:101B4000802113606B460422C905086807331042E0
:101B500028D080210422C905C86810422ED08021D7
:101B60002020C905CA688243CA6014221A701A78F4
:101B7000002A2FD18021C905C86820320243CA60DB
:101B800014221A701A78002A28D11A4B1A7D22784A
:101B90005A601D221A705932DA6013BD1A6816494C
:101BA0000A40C5E7086802430A6014221A701A78CE
:101BB000002ACED01A78013AD2B2F7E7C8680243B9
:101BC000CA6014221A7019784A1ED2B21A700029FB
:101BD000F9D1C4E71A78013AD2B2C7E71A78013AC4
:101BE000D2B2CEE72C46FF1FF446FF1F3CF0004068
:101BF0002446FF1F00200040FFFFFEFF564B70B53C
:101C00001B68012B03D1554A936D0133936502F094
:101C10007FF9534B534A1860534B544C1A600123BD
:101C2000534A1360534A13602378002B06D00622D0
:101C30005149524802F07CFA00232370504A514B1C
:101C400010681B78C1B2002B0ED14F4CC0B2237864
:101C50005BB2002B4FDB237824785BB264B21B04A9
:101C600024021B191B1813600B1C50294ED950233A
:101C7000464A47491078DBB2FF2202284BD1086858
:101C8000444C454D267890432A78964254D9227880
:101C900024782E78023B5D10A31B6B435201D31AAC
:101CA00010335B111843086002F08AFA031F012BFE
:101CB00045D83A4B1B78002B06D0394B1B78002BAC
:101CC00002D0002002F0A4F8A122364B92009978AD
:101CD000354B4A431B689B18832292009B181B7844
:101CE000033B012B03D8AF20400002F099FA0122F8
:101CF0002E4BDA8270BD237824785BB264B2FF3356
:101D0000FF341B0424021B190138ABE7CAB2022AB4
:101D1000AED20223ACE70868254C264D26789043C6
:101D20002A78964208D9227824782D78023B5B10D5
:101D3000641B63435201B2E72378DBB2B2E70228A7
:101D4000D5D11D4B1B78013B022B03D91B4B1B78B4
:101D5000022BCCD16C20C8E79809FF1FFC0FFF1F96
:101D60002867FF1FFF3F0000141003402C67FF1F70
:101D70000C10034000100340D50BFF1F7211FF1F12
:101D8000B40003408C09FF1F680AFF1F490AFF1FA8
:101D900094000340460AFF1F470AFF1FF908FF1F70
:101DA0002209FF1F300DFF1F3409FF1FBC0BFF1F4F
:101DB000440AFF1F450AFF1F1C09FF1F2309FF1FBD
:101DC00010B502F02DF90022014B1A8010BDC0465B
:101DD0002467FF1F10B502F07BFAA121054A890094
:101DE0009478054A61431268044B5218528C1A8049
:101DF00010BDC046300DFF1F3409FF1F2467FF1FB1
:101E000010B50D4B0D4A9978A1239B004B431268E6
:101E1000D218531DD97F0A4B1B88994209D2441C02
:101E200007D0C82805D0D2695B1A5A43054B5343E3
:101E3000C01802F0CDF810BD300DFF1F3409FF1F90
:101E40002467FF1F7102000070B5244D2B68002B22
:101E500028D002F045FA2B68D8402B680400002BEC
:101E600027D002F01DF92B68D8401D4B1D4A9978E8
:101E7000A1239B004B431268D118D25C91239B0095
:101E8000002A20D0CA580132CA50174B17491B6884
:101E90000868834214D3D23B181A012A1AD0144B73
:101EA000186070BD02F01CFA124B196802F038F984
:101EB000D3E702F0F5F80F4B196802F031F9D4E7D7
:101EC0000D495B18E8E7CA500C4B1B68DB68E41847
:101ED000201AE4E7F530FF30E1E7C0461C08FF1F99
:101EE000300DFF1F3409FF1F9C09FF1F2867FF1FCC
:101EF000A009FF1F1808FF1F2DFF3F003067FF1FBD
:101F000070B504000D00282916D10300A433C2883F
:101F10001B889B1A0B4A9BB293420DD906006A3666
:101F200005223100653001F0BBFF002804D13100EB
:101F3000200002F04DF970BD2900200002F0E0F908
:101F4000F9E7C046FE7F0000F8B50400012001F06B
:101F5000B7FF02F0FDF8174A17491060174D03004C
:101F6000886A174E28607568AC46164D2F680025A4
:101F7000BC4501D275687D1B134E00193560C862DF
:101F8000A4204C6A40032043486210490978002984
:101F900005D00F490978022902D10F3B1360F8BD23
:101FA000012901D1083BF9E7032901D1053BF5E7F8
:101FB000033BF3E7E408FF1F00F00040340AFF1F73
:101FC00028100040180AFF1F1C0AFF1F1C09FF1FD2
:101FD0004A0AFF1F70B580241025E405A3682B432F
:101FE000A36001F07DFFA368AB43A36070BD000058
:101FF000F7B5160080221C001023D20501919168CC
:1020000005000B43936000225A4BD7301A6002F050
:102010007FF89D232A002F009B00EB58CA32012134
:102020000092FC37002B01D00021009A386801F0A3
:102030008FFF2900009BCB311A784F4BD3351A60A4
:102040004B780A781B0213438A7812041A43CB7820
:102050001B061343494A1BBA13604B790A791B02CA
:1020600013438A7912041A43CB7931001B061343B8
:10207000434A1BBA13606B782A781B021343AA7871
:1020800012041A43EB781B0613433E4A1BBA136033
:10209000019A330213433C4A13603C4B22001B1B42
:1020A0009C4603293DDCB3089A0013005142B21A42
:1020B000032A46D1354AE018511A82784078120432
:1020C00000020243E05C043302430A600022FF2B5B
:1020D0004BDDF0222E4B12011A600F222D4B1A609D
:1020E0002D4A1368002BFCD00023224A2749136095
:1020F000091B321D0B191B68043A180A2370607003
:10210000180C1B0EA070E3700434002AF2DC80224D
:1021100010213B68D20501333B6093688B43936089
:10212000F7BD6346D578981893782D061B042B438A
:10213000157804392B43557804322D022B43036064
:10214000AFE7022A0AD1114AE05C511AE21852782C
:10215000120202430A6004339BB2B7E7012AB5D1E9
:102160000A4A521AE15C1160F5E7084959180A60F9
:102170000433ACE7000004403C0004403800044055
:1021800034000440300004400C00044000010440CE
:10219000040004401000044014000440F7B515008A
:1021A00080221C001023D2050091916807000B4388
:1021B00093600023654AD730136001F0A9FF9D2387
:1021C0003E009B00F9583B00CA363200FC33002920
:1021D00000D07FE0586801F0BBFE390032785C4BDC
:1021E000CB311A604B780A781B0213438A78AC46CD
:1021F00012041A43CB78281D1B061343554A1BBAF9
:1022000013604B790A791B0213438A7912041A432B
:10221000CB791B061343504A1BBA13604B7A0A7AD8
:102220001B0213438A7A12041A43CB7A21001B063D
:1022300013434A4A1BBA1360009A2B021343484ABD
:1022400013602200474B1B1B0093009BCE785B184A
:1022500001938B7836061B0433430E7804383343DE
:102260004E78043136023343019E33600328ECDCA0
:102270000321A808431C9B002940800003292BD17F
:102280003849E5185E18A9786D78E35C09042D02D9
:10229000294319433160030008330021FF2B2DDD52
:1022A000314B324919600F21314B19600123274905
:1022B0000B60304B19680029FCD006211B680B40CD
:1022C000042B20D080220020D20593680A318B4352
:1022D0009360FEBD01217DE7022908D121495D18E7
:1022E000E1184978E35C090219432960D3E7012921
:1022F000D3D11C495918E35C0B60CCE71948181876
:1023000001600433CAE7002310490B606346002BC9
:102310000CDC3B00FC335A68102101325A608022E9
:10232000D205936801208B439360D2E7009B9B18F2
:102330001B68190A13705170190C1B0ED3700423FB
:102340005B4291709C440432E0E7C04600000440C8
:102350003C00044038000440340004403000044095
:102360000C0004400001044004000440080F000079
:10237000100004401400044070B5061E19D002225B
:10238000614B9B799343012B13D1604B1A78FF2A41
:102390000FD15A78FF2A0CD19A78FF2A09D1DA781E
:1023A000FF2A06D11A79FF2A03D15B79FF2B00D1CE
:1023B000A7E0574B0C201A78012A08D00022554D6F
:1023C0001A702B781A00093A042A01D8212070BD0E
:1023D0005A1F012AFAD94C4CA07B042800D990E05E
:1023E000A279032A00D98CE0821E012A03D86288D0
:1023F0001F2A00D885E0002E61D0012E00D080E099
:10240000A288012AE2D0002B0AD10138032803D880
:1024100001F0D8FC151D19151F202E7001F070FD5C
:102420002B785A1E032A16D800253B4B1D60282303
:10243000237501F0FDFEA8422ED0A580C6E7022339
:1024400020202B70EAE7042322202B70E6E70323E9
:1024500021202B70E2E7073B012BB7D82F4B1B68DD
:10246000DB6A9B06B2D52E4B1A78002AAED1A27B2E
:10247000911E012901D9002AA8D1022280211A70B7
:102480002823284D89012878237501F011FE802129
:102490002878890101F014FF0123A380224B1B78C7
:1024A000002B0AD0FA228021204B92001B880902BF
:1024B0005A431C4B187801F01BFF002087E701F0FE
:1024C0009FFC2B78A680073B012B06D918482E705D
:1024D00001F0C6FE1E2001F013FD114B114C1A78BD
:1024E000002A06D080210022207889011A7001F08C
:1024F000DFFD01F0ADFD80212078090201F0D8FD5B
:10250000DBE7122063E7C046A60BFF1F6B09FF1F26
:102510001A09FF1F1C09FF1F4809FF1F3067FF1F13
:102520002309FF1F1B09FF1F2109FF1F2C09FF1F84
:102530000010004010B5002901D001F039FE10BD97
:10254000F7B5604B01919978A1239B004B435E4AFC
:10255000060014681022E418D6235B00E0583623E6
:10256000FF33E35C00279343222B41D1574B0F3AB3
:102570001A600760012501F0BBFD019B1880E8236C
:102580005B00E35C002B01D0B34258DD0023504FC9
:10259000FB70AD33FF33E3581A68002A03D09B88E1
:1025A000DB439B071DD03823FF33E35C002B18D09F
:1025B0009B235B00E35C002B13D1D133FF33E35C3F
:1025C000B3420EDAA4235B00E15AE018090A023193
:1025D00001F0DEFC23000122FE33013E01351A87A3
:1025E000FA70E8235B00E35C002B2AD0A8B2FEBDA2
:1025F00003683D00002BBED081880430090A0231F7
:1026000001F0C6FCD6235B00E3581F60B2E723004D
:10261000B133BA00FF339858013781880430090A72
:10262000023101F0B5FCE8235B00E35CBB42EEDC69
:10263000E822F61AED1800235200A354A6E700275B
:10264000F1E7200001F02CFE00281FD0002E1DDD38
:102650007319882647190193B600200001F040FD48
:102660005A30800020184068013581880430090AFA
:10267000023101F08DFC200001F0DAFCA359013396
:10268000A351BD4202D0019B9D42E6D1114BE35CB8
:10269000002BABD095239B00E35C002BA6D00E4B08
:1026A000E15A0029A2D00D4AA35C994202D9013314
:1026B000A3549BE700231A212000A35401F098FDA6
:1026C00094E7C046300DFF1F3409FF1F001403407C
:1026D000E010FF1F5A020000720200005E020000BC
:1026E000F8B51D4B1D4F1A78002A10D1BA7B002A6D
:1026F00002D101321A7003E0032AFAD0022AF8D07C
:1027000001F096FD00220120154B1A70F8BD154B03
:10271000154D1C68154B9E7801232B702878C0B28C
:1027200000F0CEFCBB7B002B0BD101F0A1FCA12360
:102730009B007343E41883239B00E41823782B70D9
:10274000E4E7032B02D101F02BFDF0E70020022B80
:10275000DCD101F075FDEAE71C09FF1FA60BFF1F86
:102760002309FF1F3409FF1F490AFF1F300DFF1FF8
:10277000F0B587B00EAD2F780FAD2D780593AC4630
:10278000634614000E4D0CAA12782E7803930D9B0D
:10279000009201932200059B029701F0E9FB2E7045
:1027A000012C01D0042C08D1802206498B88934348
:1027B000054A1278D20113438B8007B0F0BDC046A2
:1027C0001C09FF1F6C11FF1F7809FF1F0B001B3B2B
:1027D00070B504003020E02B0DD81300E025493BF4
:1027E000FF3B9BB2ED00AB4205D8034B20001982A2
:1027F0005A8201F0BDFC70BD8410FF1F10B501F0BE
:1028000087FB054B00205B68052B04D9034A5268FF
:10281000D20200D4980810BD00100040FCE100E096
:1028200070B501F0EDFA0D4B1B68FC33DC691D6AD5
:10283000FFF7E4FF6419844204D2094B01241B68AA
:10284000002B07D004220024064B1A70064A936915
:102850000133936101F0FCFB200070BD3067FF1F66
:102860009809FF1F2309FF1FFC0FFF1F70B50C4DB8
:102870002B68FC335C6A01F0C3FAFFF7BFFF2B68DB
:102880000025FC339B6AE318834204D2054B1B6886
:10289000AB4200D1051B01F0DBFB280070BDC04638
:1028A0003067FF1F9809FF1FD722044B92009B58E7
:1028B00010B5002B00D0984710BDC0460000FF1F88
:1028C000F0B587B001F008FAFFF7EEFFC54BC64C34
:1028D00004931B78022B45D1C44B1B68186A01F086
:1028E000EFFAC34BC34A1A60C34BC44A1A60A02212
:1028F000C34B52001A60049B187801F0C1FAC14919
:10290000C14801F09DFAC149C14801F099FA10226D
:10291000C04BFF201A60802252031A60802292036B
:102920001A60802212041A6001F072FA012001F08C
:1029300037FBFA20400001F0FBFA582001F070FC50
:10294000B54801F055FA012001F0C2FA072001F064
:1029500057FCE26DB14B1A4084235B001343E365DF
:1029600007B0F0BD01F0B4FBAD4E0290322001F093
:10297000A7FA33681B0628D43C2001F0A1FA0F20E7
:1029800001F09EFA974B1B78012B00D113E18025B3
:1029900033682B4200D0A1E0636C03202B436364B7
:1029A00001F08EFA01F094FB029B0299C31A5A1EA1
:1029B000814200D81A009B4B1A608C4B19681E2369
:1029C0005343994A9B18CB618BE701F081FB80232D
:1029D000E26BDB0213430390E363E26D8F4B032052
:1029E0001A4028231343E36501F06AFA0320A56E19
:1029F00001F066FAA36E0320DB03DB0B019301F009
:102A00005FFAA76EED03FF03ED0BFF0B874AAB18D0
:102A1000C22B2ED8019B9B18C22B2AD8BB18C22BC5
:102A200027D8019B2A009D4200D21A00019B9D429B
:102A300000D91D003B00974200D21300BD4200D9CF
:102A40003D005B1B122B14D80C22336814209343D7
:102A500033603368764A1340336001F031FA08215D
:102A6000A36EE26DDB038A43E265724ADB0B1360FF
:102A700085E7032001F024FAA36EDB03DB0B05934B
:102A800001F026FB039B0399C21A531E814200D812
:102A90001300694A93421BD9FF23356864492D0A04
:102AA0001D4032686B1C1B060A401B0C134333602D
:102AB0000C23326800209A43083B1343336001F033
:102AC0004FFB5E485E4BA840984205DCFEF73AFF9C
:102AD000019D0197059F99E75A48F7E700235A4E51
:102AE00033608023226CDB0213432364636C032076
:102AF0002B43636401F0E4F93368013333608023CE
:102B0000626C5B021343636405230193E26D434BE4
:102B100003201A404D4B1343E36501F0D1F908211E
:102B2000A26EE36D434F8B43E3653B6802394B4331
:102B3000D203D20B9A420CD89B1A3B2B0BD8E36DD5
:102B400043490B40E365636C0B406364414B1A607F
:102B500028E7D31AF1E7019B013BDBB20193002B7D
:102B6000D4D1E36D3A4A1340E365636C1340636468
:102B70003368042B07D9BFF34F8F374B374ADA60DE
:102B8000BFF34F8FFEE7636C0320AB43636401F038
:102B900097F9E26D214B03201A4028231343E36584
:102BA00001F08EF90822A36EDB03DB0B3B60E36DC3
:102BB0009343E3659AE70722E36B1340012B02D1AD
:102BC000002001F05DF9264D264AAB680220134033
:102BD000AB6001F075F98023AA685B001343AB601A
:102BE000E0E6C0464A0AFF1F00F000403067FF1FC2
:102BF000000003400180063DBC0003403408000093
:102C0000A40003407102000014100040FFFF3F00C9
:102C10002810004000E100E03075000000FEFEFFDB
:102C2000C4F000401867FF1F7206000091FCFFFF10
:102C3000FF00FFFF2067FF1FE30C0000E88000009B
:102C40005F361E0060361E009045FF1F2800010001
:102C5000FFFFFEFF1C67FF1F00ED00E00400FA0508
:102C60003CF00040FFFEFFFF694E336888331B686D
:102C700083F3088801F0F4F900F018FC654B664A0C
:102C80001B68934207D0002001F06AFA0221634AD0
:102C900013688B431360FFF713FE614B614C187888
:102CA000C0B201F0F5F80023A3600233A3605E4BCD
:102CB0000120236001F004F90323A36001F008FA66
:102CC000040001F025F9050001F002FA574B1860E5
:102CD00001F0C6F8564B1968621A531EA14200D281
:102CE00013008022D203934201D39B029B0A3268D5
:102CF000D16AC90700D478E04E491C0C09689BB220
:102D00004C4359432402090A641803274A49FC32F8
:102D100093680A6849489B1A494A4A4E12684A49C8
:102D20009B18414A34609A183B400193036892080B
:102D30009C46019B0A6063440360042B03D9013263
:102D40003B400A6003600B684049E418200001F032
:102D5000E7F93F4F3D493B68C3183B6020000193B2
:102D600001F0A6F83B4C20680818384920608842DA
:102D700005D9019B01333B6001F09AF8216001F015
:102D800037F9354B1B78002B0ED001F0C1F83168B4
:102D9000324B4A1B1B6812189A4233D2591A4919EE
:102DA000091A2F4801F04CF82E4C237A002B0FD033
:102DB00001F0AEF83168E3684A1B1218934224D937
:102DC000591A4919091A284801F03AF800232372C0
:102DD000264B83F3088801F0D3F8022001F090F825
:102DE000002001F0BDF901F083F8DC019900023404
:102DF000641A5900641A09214B438033CB40A4085C
:102E0000E41882E7FA218900CBE71949DBE7C046DD
:102E10003067FF1F0C0AFF1FB6412103100000405E
:102E2000490AFF1F14100040C4090000100AFF1FC8
:102E3000340AFF1F380AFF1F200AFF1F280AFF1F3E
:102E40001C0AFF1F1467FF1F240AFF1F71020000E6
:102E50006008FF1F2C0AFF1F1C09FF1FE408FF1F4B
:102E600000100040740BFF1F3C10004000000020C9
:102E7000DC050000A022054B92009B5810B5002BEA
:102E800001D0984710BD01F04BF8FBE70000FF1F91
:102E9000A122054B92009B5810B5002B01D09847FA
:102EA00010BD01F03DF8FBE70000FF1FA222054B1B
:102EB00092009B5810B5002B01D0984710BD01F02F
:102EC0002FF8FBE70000FF1FA322054B92009B5841
:102ED00010B5002B01D0984710BD01F021F8FBE799
:102EE0000000FF1FA422054B92009B5810B5002B39
:102EF00001D0984710BD01F013F8FBE70000FF1F59
:102F000070B501F005F8514B1860042000F0F8FF8F
:102F100001F09EF90400C30702D401F0F1F870BD7E
:102F200000224B4B1A604B4B1878013804282CD8E0
:102F300000F048FF03231B1F2700200001F060F86A
:102F40000128ECD0444C2378042B71D101F0E8F92E
:102F5000002806D001F08CF9582001F061F9022315
:102F60002370032000F0CCFFD9E7200001F088F89F
:102F7000E6E7200001F04CF8E2E7200001F088F8D5
:102F8000DEE7200001F084F9DAE701F019F9050025
:102F9000012808D1314B1B78053B012B03D82000B9
:102FA000FFF768FFCEE72C4B1B78022B01D0052BD7
:102FB00020D1022D28D12A4B9B7BAB431CD1200072
:102FC000FFF766FF254B18780128BBD16405B9D4FB
:102FD000234925224B7B034205D1233A13405A4211
:102FE000534126331A000B7D9342ABD9322000F0B7
:102FF000E7FFA7E7022D07D1184B1B78052B11D14E
:103000002000FFF753FFDDE7012D0BD1012B03D18A
:103010002000FFF759FF95E7062B03D12000FFF7AB
:1030200061FF8FE7200000F07BFF022D8AD1C9E706
:10303000032B04D10B4B987C00F0BAFF91E7072BD0
:103040008FD1094B987B01F01BF98AE79C09FF1F80
:103050009809FF1F9009FF1F2309FF1F1C09FF1F6D
:10306000A60BFF1FBC0BFF1FD40BFF1FFA210A4B3F
:103070000A4A49001A640A4A5A500A4A04395A50FC
:10308000094A08319A64094A5A50094A5C315A502F
:10309000084ADA667047C0460000FF1F7127FF1F0D
:1030A0006D28FF1F2128FF1F7923FF1FE126FF1F27
:1030B000011EFF1FD51DFF1F10B500F06BFE10BDD8
:1030C0008023F7B59C46264B264F01932649274A75
:1030D000274D284C284B02281AD1604638600868D2
:1030E000264E304080263603304308600199097827
:1030F000002909D11660224A2A60224A2260E02271
:1031000019689143A03A1BE08021C9021160F2E7DF
:1031100066463E600F68194E3E408027FF023E43E0
:103120000E600199097800290DD1176001280ED190
:10313000154A2A60154A2260E02219689143C03A74
:103140000A431A60F7BD802189021160EEE7E02191
:103150000F4A02432A600F4A22601A688A43F0E746
:103160004B0AFF1FE0000340D800034090000340DB
:10317000000003405000034040000340FFFFE3FF16
:103180000280063D804508220180063D80660822B7
:103190000080069880550822F8B51E4B80261A68D4
:1031A000002014003440324232D11A681A4F3243A0
:1031B0001A6001223B68063093433B6000F080FEBA
:1031C0000122164D2B681E432E603B680A261343CE
:1031D0003B608027BF00124B1B683B4211D1013E70
:1031E000F6B2FF2E09D17E220E4B1C682B68E40B31
:1031F0001440934323432B6005E0082000F060FE59
:10320000E9E7002EEFD180222B68600893432B6002
:10321000F8BDC046C4F000405CF0004018F000402B
:1032200068F0004060F0004010B500F049FF012157
:103230005820034A00F0ACFFFFF7AEFF10BDC046B8
:10324000600AFF1F10B578220021034800F0E0FF5C
:1032500000F00EFE002010BD386AFF1F70B504009C
:1032600000F0CEFD00230C200B4A010059438D18BD
:10327000515C00290DD0A14208D1012300246B70BC
:1032800000F05EFF00F0E4FE200070BD01330A2B69
:10329000EBD11224F6E7C046386AFF1F70B5040070
:1032A00000F0AEFD002319001D000D4A1078002823
:1032B00006D0A0420CD1557001310C320A29F5D14B
:1032C000002B0AD100F0D4FD00F0C2FE002070BD3A
:1032D0005078461EB0411B18EEE700F031FFF3E7CF
:1032E000386AFF1FF7B504000C20002384460E4DFA
:1032F000019267465F43E85D7E19A04212D0002824
:103300000BD10A4B9C4662461B7808331370019B15
:1033100070707C557160B360FEBD01330A2BE8D13B
:103320000320F9E70720F7E7386AFF1F346AFF1F19
:103330008020F8B5484BC0051B68C1248360474B0B
:10334000FF251A68012313434361454BA4001A6803
:10335000444B40211A60444B1A68444B1A60444B5A
:103360001A59AA431A51C52292009E58AE433143BE
:10337000802699509F583F49F6010F403E439E508A
:103380009E5880273602360A3043985080201A59BA
:1033900000020A4002431A5104341A59364E3F04BF
:1033A000324080263A431A511A5936061202120A3E
:1033B00032431A5108341A5980260A4002431A51DE
:1033C000C32292009F58B446AF4337439F509F5843
:1033D000294E0F4007439F509F58374080263604A0
:1033E000374380269F509F5836063F023F0A374397
:1033F0009F50C0221F59AF433A431A511A59120223
:10340000120A1643C6221E5192009C58AC436546D0
:103410002C439C509C5800250C4020439850C720BA
:1034200080001A58154C1140C02212020A431A504B
:10343000134B1B78DB08AB4201DC0020F8BD23787E
:10344000002B06D0A368002B00D0984701350C3420
:10345000EEE71220F2E7C0462846FF1F2446FF1F72
:10346000B0F00040306AFF1FB4F000402C6AFF1F2C
:1034700000E100E0FF00FFFFFFFF00FF386AFF1FD1
:10348000346AFF1F030010B51F2809D80722002047
:103490001340072404490A78A24313430B7010BD5C
:1034A00000230620F5E7C046346AFF1F034A04499B
:1034B000136800200B4013607047C0461CF00040AA
:1034C000FFFFC1FF054B06491B780A6805485B07EB
:1034D00002401B0B134300200B607047346AFF1F30
:1034E0001CF00040FFFFC1FF70B50C25FFF7EAFF9D
:1034F0000A4B1C780A4BE4086543ED18002C01D1F7
:10350000200070BD2B78002B06D06B68002B00D0FC
:103510009847013C0C3DF1E71220F2E7346AFF1FA7
:103520002C6AFF1F1FB5002102220B0001910091A0
:10353000052000F005FD02230B490A681A42FCD160
:1035400020230393039B5A1E0392002BFAD1074AB0
:103550001368002BFCDA0B246C442000012100F0DE
:103560003FFE207804B010BD90C8004000C8004065
:1035700013B504000A4B0193019B002B01D11120CC
:1035800016BDFFF7CFFF23000340044205D00520FE
:1035900000F096FC019B013BEDE71800F0E7C04608
:1035A000FFFFFF0707B500F02BFC80220821D205A2
:1035B000936A0191002B01D10739916202210C4AD3
:1035C00011600199481E01900029FAD10331116060
:1035D000053101910199481E01900029FAD111602D
:1035E000002B02D18022D205936200F031FD07BD8D
:1035F00000C00040F0B52D4C89B02378002B4FD18E
:10360000FEF780F902232A4F03903A681A42FCD150
:1036100020230693069B5A1E0692002BFAD1254EB4
:103620003368002BFCDA0120FFF7A2FF011E02D055
:10363000112009B0F0BD030003220190009005ADF8
:103640009F2000F07DFC0321280000F0C9FD02232B
:103650003A681A42FCD120230793079B5A1E07920F
:10366000002BFAD13368002BFCDA0120FFF780FF32
:103670000028DDD10398FEF759F9AA786B78110478
:103680001B020B4329780B4363601300113B0A496B
:10369000052B07D801239340A3600B6001232370FF
:1036A0000020C6E780231B03F6E7C0461046FF1F35
:1036B00090C8004000C800409808FF1F1E4B30B55E
:1036C0005A6818781D4B85B0D31859424B410121D7
:1036D0000093002300F044FC194B1A4A02259A6318
:1036E00000221A6510325A658022C4219D65164B4E
:1036F0001648D202DA6789004258154B80241A40D6
:1037000080231B0413434350642341200393E405A7
:1037100000F006FA402000F003FA6562039D6B1E7C
:103720000393002DFAD103236362FFF73BFFA562E9
:10373000FFF760FF05B030BD1C46FF1F95FFFEF789
:1037400000C80040050001FF04E100E000E100E0E6
:10375000FFFF00FFF0B585B00700FEF7D3F80223A6
:1037600005002D4C22681A42FCD120230093009BB7
:103770005A1E0092002BFAD1284E3368002BFCDA37
:103780000120FFF7F5FE002803D01124200005B02A
:10379000F0BD234B2360022322681A42FCD1202370
:1037A0000193019B5A1E0192002BFAD13368002B22
:1037B000FCDA0120FFF7DCFE0028E6D1194B1F6080
:1037C000022322681A42FCD120230293029B5A1E34
:1037D0000292002BFAD13368002BFCDA0120FFF7AC
:1037E000C7FE0028D1D1104B2360022322681A4261
:1037F000FCD120230393039B5A1E0392002BFAD182
:103800003368002BFCDA0120FFF7B2FE041EBCD1A6
:103810002800FEF78BF8B9E790C8004000C80040C8
:1038200001000006A8C800400180000110B500207A
:10383000FFF790FF10BD000010B5064B18705960DF
:10384000FFF73CFF00211320034AFFF74BFD002048
:1038500010BDC0461C46FF1FBD36FF1FF0B504005B
:1038600085B003920291FEF74DF8882263035B0B4B
:1038700052051A438023DB059D6A8023274F00925F
:10388000BA68002601901B039A420CD9F82326003F
:103890001B041E401C4206D08022214B52025E6255
:1038A00019680A431A60002D0BD100F0A9FA022210
:1038B0001C4B1A608023DB055A62013A9A6200F0C1
:1038C000C7FB0023039A934220D1002D0AD100F0B8
:1038D00097FA144B03221D608023DB055A629D6218
:1038E00000F0B6FB8023BA681B039A4208D9002E69
:1038F00006D000220A4B0C495A621A680A401A6024
:103900000198FEF713F8002005B0F0BD009A029967
:10391000D2181278CA540133D4E7C0461046FF1FAC
:1039200000C8004000C00040FFFFFEFFF0B587B0B8
:10393000029103920400FDF7E5FF019000F060FAA8
:10394000802302250122234EDB0535605D629A62E9
:1039500000F07EFB204F3B682B42FCD120230493D8
:10396000049B5A1E0492002BFAD11C4D2B68002B8D
:10397000FCDA0120FFF7FCFD002802D0112007B07F
:10398000F0BD2000039A029900F052FA02230400CD
:103990003A681A42FCD120230593059B5A1E0592D2
:1039A000002BFAD12B68002BFCDA0120FFF7E0FD99
:1039B000051EE3D100F024FA80230322DB053560E5
:1039C0005A629D6200F044FB0198FDF7AFFFE0B240
:1039D000D5E7C04600C0004090C8004000C8004085
:1039E000F0B5802489B00600FDF78CFFE405A36ADA
:1039F00002250393029000F003FA0123304F3D604B
:103A00006562A36200F024FB2E4C23682B42FCD19C
:103A100020230593059B5A1E0592002BFAD12A4DAF
:103A20002B68002BFCDA0120FFF7A2FD002803D051
:103A30001124200009B0F0BD244B2360022322682A
:103A40001A42FCD120230693069B5A1E0692002B95
:103A5000FAD12B68002BFCDA0120FFF789FD021E4A
:103A6000E6D11B4B03211E60030001900090202033
:103A700000F066FA022322681A42FCD12023079341
:103A8000079B5A1E0792002BFAD12B68002BFCDAF9
:103A90000320FFF76DFD041ECAD100F0B1F98023A9
:103AA0000322DB053C605A629C6200F0D1FA039B62
:103AB000002B01D1FFF776FD0298FDF737FFB8E73D
:103AC00000C0004090C8004000C80040010000064F
:103AD00094C8004007B5000201910422000A01A920
:103AE000FFF724FF0EBD000073B5050005240B4A47
:103AF000A3005B429B1819686B46DE1D300000F086
:103B0000A7F9022804D133782B55013CEFD276BDBA
:103B1000052CFCD00128FAD10230F8E71409001175
:103B20001F2807D8012380228340D20591680B43C8
:103B3000936070473F2808D80123802220388340B3
:103B4000D20551690B435361F3E75F28F1D8012394
:103B5000802240388340D205116A0B431362E8E7A4
:103B60001F2807D8012280218240C9058B68934312
:103B70008B6070473F2808D801228021203882407E
:103B8000C9054B6993434B61F3E75F28F1D80122E4
:103B9000802140388240C9050B6A93430B62E8E7F5
:103BA0001F2810D880230200DB05153A1968012A66
:103BB00006D820229143196019680A431A60704799
:103BC00001228240F6E73F2811D880230200DB055E
:103BD000353AD968032A06D810229143D960D968AA
:103BE0000A43DA60EBE7012220388240F5E75F28DC
:103BF000E5D842238022181A413B8340D205516AFE
:103C000099435162516A0B435362D8E710B50400DF
:103C1000012813D1A022184992050B685B015B09AA
:103C200013430B60154B164A19681140154A0A4395
:103C30001A60402219680A431A6010BD0028FCD19E
:103C400001000A2000F0CCF921000B2000F0C8F997
:103C5000C0220A4B920019680A4340211A601A6870
:103C60008A431A60B022044912060B685B015B09A3
:103C700013430B60E1E7C04614F000401CF0004025
:103C80007F00FEFF80FD010072B6074A1368013312
:103C900013600422054B1A600023054A136080223A
:103CA000D2055360FEE7C0467808FF1FC0F0004011
:103CB000C4F00040044B054A1A60054B1A6000220C
:103CC000044B1A607047C046140AFF1F841E000090
:103CD000380AFF1FC4F000400023034A1360034A60
:103CE0001360034A1360704754F0004040F10040F5
:103CF00044F10040002310B5184C8AB000930193A2
:103D00002378012B27D06946012000F099F900287B
:103D100017D1009B12490293019B06AA0393114BF2
:103D200002A81B680493104B1B68059300F0D8F899
:103D300010220E4906A800F0B3F8002804D1FF2392
:103D4000237000200AB010BD0123094A074902A8C8
:103D5000237000F0C5F80120F4E7C0463467FF1F68
:103D600010290011082900110C2900112029001127
:103D70003867FF1F13B501246946012000F060F980
:103D8000034B00940193FFF7B5FF200016BDC0461A
:103D9000BB0B000010B5FFF79FFFFFF7EBFF0028FC
:103DA00002D0024B984710BDFEE7C046E1A20000DA
:103DB00002B4714649084900095649008E4402BCC4
:103DC0007047C04602B4714649084900095C490081
:103DD0008E4402BC7047C04603B471464908400097
:103DE0004900095A49008E4403BC70470000000096
:103DF00001B40248844601BC604700BF8D11010038
:103E000001B40248844601BC604700BF75A90000A8
:103E100001B40248844601BC604700BFED6B01005D
:103E200001B40248844601BC604700BFE927000096
:103E300001B40248844601BC604700BF957301008D
:103E400001B40248844601BC604700BF2D6C0100EC
:103E500001B40248844601BC604700BF9938001194
:103E600001B40248844601BC604700BFC16601003E
:103E700001B40248844601BC604700BFADAE0000FB
:103E800001B40248844601BC604700BFEDA50000B4
:103E900001B40248844601BC604700BF8914010098
:103EA00001B40248844601BC604700BFCD4C01000C
:103EB00001B40248844601BC604700BF090E0000FF
:103EC00001B40248844601BC604700BF018900007C
:103ED00001B40248844601BC604700BFE5120100FE
:103EE00001B40248844601BC604700BFDD3F0000CA
:103EF00001B40248844601BC604700BF85520100FE
:103F000001B40248844601BC604700BF19070100A4
:103F100001B40248844601BC604700BFC95C01008F
:103F200001B40248844601BC604700BFE9170100A4
:103F300001B40248844601BC604700BF85120100FD
:103F400001B40248844601BC604700BF496D0100CE
:103F500001B40248844601BC604700BF2144000010
:103F600001B40248844601BC604700BFC56D010032
:103F700001B40248844601BC604700BF9D6A00004E
:103F800001B40248844601BC604700BF7997000035
:103F900001B40248844601BC604700BFC11501005E
:103FA00001B40248844601BC604700BF69110100AA
:103FB00001B40248844601BC604700BF4DF90000CF
:103FC00001B40248844601BC604700BF613701006C
:103FD00001B40248844601BC604700BF8937010034
:103FE00001B40248844601BC604700BFD59F001160
:103FF00001B40248844601BC604700BFD5440100BB
:1040000001B40248844601BC604700BF013401008E
:1040100001B40248844601BC604700BF053401007A
:1040200001B40248844601BC604700BF8D82000095
:1040300001B40248844601BC604700BF59760100C4
:1040400001B40248844601BC604700BFE1AC0000F7
:1040500001B40248844601BC604700BF9DA900002E
:1040600001B40248844601BC604700BFC9A90000F2
:1040700001B40248844601BC604700BFE9F6000075
:1040800001B40248844601BC604700BF0934010006
:1040900001B40248844601BC604700BFF535010009
:1040A00001B40248844601BC604700BF6D0B0100AB
:1040B00001B40248844601BC604700BFB35201000E
:1040C00001B40248844601BC604700BFED680100AE
:1040D00001B40248844601BC604700BF156B010073
:1040E00001B40248844601BC604700BFD9B000005B
:1040F00001B40248844601BC604700BFCD0C0100FA
:1041000001B40248844601BC604700BFDD0A0100DB
:1041100001B40248844601BC604700BF89440000E6
:1041200001B40248844601BC604700BF090E00008C
:1041300001B40248844601BC604700BFE94C01005D
:1041400001B40248844601BC604700BF21A90000B9
:1041500001B40248844601BC604700BFBD5C010059
:1041600001B40248844601BC604700BF016C0100F5
:1041700001B40248844601BC604700BF116E0000D4
:1041800001B40248844601BC604700BFA1AF0000F3
:1041900001B40248844601BC604700BF01670100CA
:1041A00001B40248844601BC604700BF75F80000B6
:1041B00001B40248844601BC604700BFE9D4000056
:1041C00001B40248844601BC604700BFDD0C010019
:1041D00001B40248844601BC604700BF85C10000AD
:1041E00001B40248844601BC604700BF3D71010034
:1041F00001B40248844601BC604700BF53B90000C7
:1042000001B40248844601BC604700BFF90D0100BB
:1042100001B40248844601BC604700BFB70E0000ED
:1042200001B40248844601BC604700BF7912010016
:1042300001B40248844601BC604700BFA9D8000011
:1042400001B40248844601BC604700BF19FA00006F
:1042500001B40248844601BC604700BFBD0B0100A9
:1042600001B40248844601BC604700BFC1A50000FC
:1042700001B40248844601BC604700BF6DF60000EF
:1042800001B40248844601BC604700BFC1F700008A
:1042900001B40248844601BC604700BFF935010003
:1042A00001B40248844601BC604700BF71B0000001
:1042B00001B40248844601BC604700BFC1B300118D
:1042C00001B40248844601BC604700BF0D520100A2
:1042D00001B40248844601BC604700BFF9ED00000C
:1042E00001B40248844601BC604700BFE90B0100ED
:1042F00001B40248844601BC604700BF8B520100F4
:1043000001B40248844601BC604700BF51B80000B8
:1043100001B40248844601BC604700BFF9A6000012
:1043200001B40248844601BC604700BF01D70000C9
:1043300002000000D2BC001101000000A8BA001168
:1043400002000000CEBC0011010000007043FF1FFE
:1043500002000000B0BA0011010000008064FF1FDD
:1043600002000000CCBC001103000000F463FF1F3A
:104370001200000002000000D2BC00110100000089
:10438000ECBA001102000000CEBC001101000000D8
:10439000E9BA001102000000F6BA001103000000A3
:1043A0002F64FF1F02000000CCBC001103000000BE
:1043B0004464FF1F02000000CEBC00110100000099
:1043C000E8BA001102000000F4BA00110300000076
:1043D0000564FF1F02000000CCBC001103000000B8
:1043E0002664FF1F02000000D2BC00110100000083
:1043F0002CBB001102000000CEBC00110100000027
:10440000B944FF1F020000003EBB00110100000084
:1044100027BB001102000000CEBC0011010000000B
:10442000B844FF1F020000003CBB00110100000067
:104430004C64FF1F02000000CEBC00110100000010
:10444000B744FF1F020000003ABB0011010000004A
:1044500017BB001102000000CEBC001101000000DB
:10446000B644FF1F0200000038BB0011010000002D
:1044700012BB001102000000CEBC001101000000C0
:10448000B544FF1F0200000036BB00110100000010
:104490000DBB001102000000CEBC001101000000A5
:1044A000B444FF1F0200000034BB001101000000F3
:1044B00008BB00110202020202020000000000001C
:1044C0000D0C0000A94C00116D4C001180BB0011B7
:1044D00090011D0018001800FFFF070102030405EA
:1044E00006020106000000000000000000000000BD
:1044F00000000000000000000000000000000000BC
:104500000300000002000000D2BC00110100000006
:1045100000BC001102000000CEBC00110100000030
:104520007445FF1F020000000ABC001101000000DA
:104530007A64FF1F02000000CCBC001103000000E1
:10454000E466FF1F02000000CEBC00110100000065
:104550007445FF1F0200000008BC001101000000AC
:104560007C64FF1F02000000CCBC001103000000AF
:10457000DC66FF1F120000000001000000000111B6
:10458000FFFF000050485936000000000000000006
:104590000100000091BB00110B000500F7000000B6
:1045A000B4000028002800283075A000A000A0005A
:1045B000A00000080008E001F0001000100010004A
:1045C00010001000100050005000500010001000AB
:1045D000D0070000000000000F000100050030754A
:1045E00007001000010081FF00000000FF00000034
:1045F000BD710011C56F0011556D0011FFFF010065
:10460000FF000000D99B0011559900116D98001111
:10461000000000000000000000000800040000008E
:104620003B0001085902E00188212800FF0000003A
:1046300002000000D2BC00110100000098BD001172
:1046400002000000CEBC001101000000AD46FF1FBB
:1046500002000000CABC001101000000F06AFF1F48
:1046600002000000CEBC001101000000AC46FF1F9C
:1046700002000000C8BC001101000000AA46FF1F94
:1046800002000000CEBC001101000000A846FF1F80
:1046900002000000C6BC001101000000A046FF1F80
:1046A000180018001D009001020000030202000023
:1046B00002000000D2BC001101000000ACBD0011DE
:1046C00002000000CEBC001101000000F046FF1FF8
:1046D00002000000C4BC0011000000000000000047
:1046E00002000000CCBC001103000000106BFF1F93
:0246F00020FFA9
:040000051FFF184180
:00000001FF
